:100000001DC2000053C2000051C200004FC20000D8
:100010004DC200004BC2000049C2000047C20000B0
:1000200045C2000043C200000C94DD2E0C94C22F88
:100030000C94EB0F3BC2000039C2000037C2000035
:1000400035C2000033C2000031C200002FC20000E0
:100050002DC200000C94B92E29C2000027C2000056
:1000600025C2000023C2000021C200001FC2000000
:100070001DC200001BC2000019C2000017C2000010
:1000800015C2000013C2000011C200000FC2000020
:100090000DC200000BC2000009C2000007C2000030
:1000A00005C2000003C2000001C2000005010902F0
:1000B000A10185020901A1000509190129081500FE
:1000C0002501950875018102050109300931158165
:1000D000257F95027508810609381581257F9501D0
:1000E00075088106050C0A38021581257F95017572
:1000F000088106C0C005010980A101850319012AF4
:10010000B700150126B700950175108100C0050CD8
:100110000901A101850419012AA002150126A002E6
:10012000950175108100C00660FF0961A101096297
:10013000150026FF00952075088102096315002629
:10014000FF00952075089102C005010906A101056F
:100150000719E029E7150025019508750181029529
:1001600001750881010507190029FF150026FF0008
:100170009506750881000508190129051500250156
:10018000950575019102950175039101C00000006C
:10019000000000000000000000000000000000005F
:1001A000000000000000000000000000000000004F
:1001B000007E0F00D4FFFFFFC700000078000000A2
:1001C00000000000002A2B280000000000000000B2
:1001D000000000000000000029000000002C1E3478
:1001E00020212224342627252E362D3738271E1F7E
:1001F000202122232425263333362E37381F0405A9
:10020000060708090A0B0C0D0E0F10111213141516
:10021000161718191A1B1C1D2F3130232D350405F4
:10022000060708090A0B0C0D0E0F101112131415F6
:10023000161718191A1B1C1D2F3130354C09025B7B
:1002400000030100A03209040000010301010009BC
:100250002111010001224400070581030800010962
:100260000401000203000000092111010001222203
:100270000007058203200001070503032000010990
:100280000402000103000000092111010001227B8A
:10029000000705840320000112010002000000088D
:1002A000435042540100010203011C03760069001F
:1002B00061006C003A0066003600340063003200D2
:1002C0006200330063000000240343006C006100FF
:1002D0007300730069006300200054007200610025
:1002E00063006B00620061006C006C0000000E0394
:1002F00050006C006F006F00700079000000040374
:100300000904D100D300D200D400D500FD377A58BB
:100310005A000004E6D6B44602002101160000008F
:10032000742FE5A3E0018800EF5D003D8889C65485
:1003300036C3174FE4E468771740EC062B597590E5
:10034000EA1B9E88D5853C2B2D4649B919FCF467DC
:10035000F3A7C15AE35727ECA65FCF01EFA012F332
:1003600075408571C8B6B71AD95082EFCEEC022C11
:100370004BF169D1ADF2D35939B7ECCF0C68A31A60
:10038000230109F1C2D35B7E87CC6DA17641DF18D2
:1003900080A47EAE025DCA7A3D0428A38325519ACB
:1003A000FF214AB537E83ED7103AB24F82E5DD9BD0
:1003B000990185D12E28DDC1DDFF435BE43FA12CEF
:1003C000C43E82271EE55CF80163364014C837E45A
:1003D000C4547DD3F980451BCBCF840E89562F02A0
:1003E000603F17246BEC672929A3A6AF9B076E908B
:1003F000BCE811B79AF314DFF8395779205B05D6BA
:10040000014BF2B2346B9D15EDBB99D53498EECB10
:100410002A711B840FF78AE71C00000079A72A4283
:100420008977A32D00018B02890300004E24F55F1C
:10043000B1C467FB020000000004595A11241FBE1A
:10044000CFEFDAE0DEBFCDBF04B603FE18C0809167
:10045000D5059091D605A091D705B091D8058730E4
:10046000904BA740B04B59F41092D5051092D60589
:100470001092D7051092D805E0E0F8E3099511E055
:10048000A0E0B1E0E6E2F9E602C005900D92A43BDF
:10049000B107D9F725E0A4EBB1E001C01D92A53D5D
:1004A000B207E1F70E943F260C941734A9CDA4E0CF
:1004B000B0E0EDE5F2E00C94A2312C01FB013A0131
:1004C00029833A830B831C831701960185017401EC
:1004D000898C9A8C808191814816590614F4518236
:1004E0004082D301CD90DC901197C414D5041CF444
:1004F0004D925C926201A080B180C6018A199B096D
:100500008A309105ECF163E070E00E94ED316A0DF4
:100510007B1D461657060CF07BC0AB81BC818C91CD
:10052000811509F470C0D7018D919C91DC01AA0F4F
:10053000BB1FA20FB31FCD92DC92D7018D919C916E
:1005400011978E3191050CF057C001968D939C93B5
:1005500040815181D3018D919C91841B950B97FD16
:10056000019695958795840F951F91838083D3017C
:100570008D939C93A981BA811C92AB81BC811C9202
:10058000AB8DBC8D8C91811509F466C0D901225CBC
:100590003F4F80E090E04D915D91840F951F2A17A9
:1005A0003B07C9F76FE170E00E94ED319B01D40178
:1005B0008C91811509F469C0F101A101425C5F4F82
:1005C00080E090E061917191860F971F4E175F0751
:1005D000C9F76FE170E00E94ED31FB01C9018E1B8C
:1005E0009F0B63E070E00E94ED31CB018E0F9F1FE7
:1005F0002496E2E10C94BE311D921C9281E0AB8DF9
:10060000BC8D8C93A5CF81E0A981BA818C93B8CFA2
:10061000641575050CF0B4CFA981BA818C91811550
:10062000B9F0D8018D919C91DC01AA0FBB1FA20DDE
:10063000B31DAD92BC92D8018D919C9111978E31D2
:1006400091050CF482CF1D921C9281E0D401D9CF88
:1006500081E0AB81BC81DACFD7016D917C91D9016A
:1006600020E030E080E090E06115710551F4D301A5
:100670002D913C919CCF4D915D91840F951F2F5FE3
:100680003F4F26173707BCF38FCFD8016D917C9170
:100690006115710581F0F10140E050E080E090E0EB
:1006A000461757070CF097CFA191B1918A0F9B1F66
:1006B0004F5F5F4FF5CF0190F081E02D8FCF9C0110
:1006C0009A9581159F4118F5F32FF270EE27832F2D
:1006D0008170732F74706627532F5870442734FF2E
:1006E0000CC08295807FEF2B09F08062672B09F0A8
:1006F0008064452B69F080680895EF2B09F08260D3
:10070000672B09F08460452B19F08860089580E01C
:100710000895CF93DF93EB01D2DFFE010995DF91BE
:10072000CF9108958093CB0508958093CC050895CB
:1007300021E030E001C0220F8A95EAF78091CC05D4
:10074000822BF3CF21E030E0A90102C0440F551FF6
:100750008A95E2F7CA0180959091CC058923E5CF6F
:10076000911121C08530F8F491E001C0990F8A956C
:10077000EAF7892FE8EEF3E040E050E070E0919175
:10078000DF019B01042E02C0369527950A94E2F7FB
:10079000217021952927282329272E934F5F5F4F0A
:1007A0004330510561F70895682F892F91111CC0BE
:1007B0006530D8F4E8EEF3E040E050E0219130E01D
:1007C000062E02C0369527950A94E2F7217033274A
:1007D000042E01C0220F0A94EAF7822B4F5F5F4F6D
:1007E0004330510559F7089580E008959091CC0564
:1007F00021E030E0F90101C0EE0F8A95EAF7D90156
:1008000002C0AA0FBB1F6A95E2F7EA2B01C0220FB4
:100810004A95EAF7892F8E23E81303C0892F822B8C
:1008200084CF2095822F8923FBCF809196039091CE
:100830009503981301C008958F5F8770FACF909148
:1008400017058095892380931705282F277021117C
:1008500010C0891771F09091CE0592FF0AC086955D
:10086000869586956FDF10921705109219051092E4
:1008700018050895982F90958091140589238093E9
:100880001405089580911305811531F01092130518
:1008900010921B0510921A050895803E9105D9F11A
:1008A000C8F48133910509F482C048F48932910576
:1008B00009F472C08A32910509F480C00895893321
:1008C0009105E9F082389105D1F08533910509F45D
:1008D0005EC00895843E9105D9F148F4823E9105A9
:1008E00039F1833E910549F181EE90E00895863E0D
:1008F0009105C9F1873E910509F43EC00895209104
:10090000CD052370211164C02091CE0523FF14C0B2
:1009100089E290E008952091CD0520FD45C03091F9
:10092000CE0530FF09C024FD24C083EE90E0089579
:100930002091CD0522FDF7CF08952091CD0522FD10
:1009400044C03091CE0530FD43C024FFF5CF11C027
:100950002091CE0521FFF0CF8091CD0584FD09C007
:1009600087EE90E008952091CD0523FFE5CF24FF89
:10097000F7CF80E090E008952091CD0523FD2BC0B6
:100980003091CE0531FFE1CF84EE90E008952091C3
:10099000CD0525FFD1CFBCCF2091CD0525FD1EC0B3
:1009A0002091CE0523FFC8CF89E390E008952091E0
:1009B000CD0526FFC1CF8AE290E008952091CD05B4
:1009C00026FFBACF81E390E0089582EE90E008958B
:1009D00080EE90E0089586EE90E0089585E390E043
:1009E00008959091CD0592FF10C041E0282F247109
:1009F000243009F040E031E0282F2871283009F038
:100A000030E0431711F02CE0822793FF10C041E043
:100A1000282F2471243109F040E031E0282F28717B
:100A2000283109F030E0431711F02CE08227309193
:100A3000CE0530FF10C051E0282F2171213009F080
:100A400050E041E0282F2871283009F040E0541789
:100A500011F029E0822731FF10C041E0282F2171D9
:100A6000213109F040E031E0282F2871283109F0C8
:100A700030E0431711F029E0822794FD877E089526
:100A80001F93CF93DF9309DFEC01811522E59207D5
:100A900008F052C0811540E5940708F0CDC0803EB3
:100AA000910520F58D3C910508F0A1C0883A91058B
:100AB00070F4853A910508F097C081309105B9F13D
:100AC0000497813A910598F1C0E0D0E030C0885A8F
:100AD00091094B97C8F7C85AD0E0CC0FDD1FC35C13
:100AE000DE4F0990D881C02DD46421C0811550E417
:100AF0009507B0F4C11580E2D80708F0B3C0C83E2E
:100B0000D105A8F0CE019A9581159F41E8F68D2F69
:100B100068DF182FCE019927C0DEEC01D12B07C06A
:100B20009927BBDECC27DF70C82BD92BD06ACE012A
:100B3000DF91CF911F910895803842E59407C8F561
:100B4000803652E5950708F05BC0C03482E5D807CF
:100B5000D0F4C03292E5D90708F04BC08C2F8695AF
:100B6000869520E2829FC0011124C37021E030E00D
:100B7000A90102C0440F551FCA95E2F7EA01C82B2C
:100B8000D92BDD68D4CF8C2F86958695877050E25F
:100B9000859FC0011124C37021E030E0A90102C08B
:100BA000440F551FCA95E2F7EA01C82BD92BDC6820
:100BB000BECF803C52E5950758F48F71C03AD245BC
:100BC000A0F590E0982F8827EC01C46FD06AAFCFD2
:100BD000805C9245809708F077CFDC2FCC27CC271C
:100BE000DF71C06FD06AA3CFA497D064A0CFD065C7
:100BF0009ECFCF71D0E0DC2FCC27C16FD06A97CFCA
:100C000086958695877020E2829FC0011124C3706B
:100C100021E030E0A90102C0440F551FCA95E2F758
:100C2000EA01C82BD92BDA6882CFDBDEC82FD0E0EF
:100C3000DC2FCC27D0627BCF8F71D3DE93E0CC0F3B
:100C4000DD1F9A95E1F7CC27DF70282F30E084FF75
:100C500005C050E1859F900111243327C22BD32B6F
:100C6000D06965CF8D2F8F71BCDE182FCE019927EB
:100C700014DEEC01D12BDECF80E0089581152CE746
:100C8000920741F42091820330918303232B11F4C6
:100C900080E090E00895EDE8F4E080E090E061E12C
:100CA00075E244E355E226EA35E2778366835187AD
:100CB000408733872287978786870196709688308A
:100CC000910599F7089510925D0510925C05ECE18D
:100CD000F5E08581811102C014821682379685E085
:100CE000E435F807B1F70895AC0130915F056091E4
:100CF0005E05232F621301C00895822F90E0FC014E
:100D0000EE0FFF1FEC5AFA4F0190F081E02DE4172F
:100D1000F50791F467E0649FF001659FF00D1124E1
:100D2000E45EFA4F41E044832313E6CF01968370DB
:100D3000992780935F0508950196282F2370DACFB5
:100D4000FC018481862381110AC082818115B9F05A
:100D50006823908593FF05C081E061110FC080E09A
:100D60000895282F22952F708F70282B962F9295FB
:100D70009F706F70962B81E02913F1CF089581E069
:100D80000895282F35EB2303C001112497FF04C0D9
:100D900080589109892F089580589F4FFBCF8091EB
:100DA000ED0380FD14C081FD14C082FD16C080914A
:100DB000EC03811581F08E3180F420E5829FC00123
:100DC00011246EE170E00E94ED31862F089584E1D8
:100DD000089588E2089588E0089580E50895809157
:100DE000ED0380FD17C081FD17C082FD19C0809101
:100DF000EB03811599F0883298F428E0829FC001B6
:100E0000112468E270E00E94ED316115710551F026
:100E1000862F089562E0FCCF64E0FACF61E0F8CF5E
:100E200068E0F6CF81E00895FA01309709F009955E
:100E30000895E0918B03F0918C03309739F0019085
:100E4000F081E02D309711F00995089580E0089524
:100E5000DC01E0918B03F0918C03309759F086818F
:100E60009781892B39F082E08C930680F781E02D01
:100E7000CD0109950895A3E0B0E0E1E4F7E00C941A
:100E8000B2319C018091DC019091DD0182179307C2
:100E9000B1F03093DD012093DC01E0918B03F09100
:100EA0008C03309761F00084F185E02D309739F0A4
:100EB00083E089833B832A83CE010196099523969B
:100EC000E2E00C94CE31A3E0B0E0E9E6F7E00C9468
:100ED000B2319C018091DA019091DB018217930776
:100EE000B1F03093DB012093DA01E0918B03F091B4
:100EF0008C03309761F00084F185E02D309739F054
:100F000084E089833B832A83CE0101960995239649
:100F1000E2E00C94CE319C01FC0132968FEF90E020
:100F20004191461751F08F3F19F4411101C0892FAB
:100F30009F5F9630A9F78F3F09F40895280F311D60
:100F400087FD3A95F90162830895E8EBF1E091910C
:100F5000891302C0DF011E9291E0EE3BF907B9F759
:100F60000895DC01FB0111969C91119781819813E2
:100F700022C012968C911297811519F092818913D3
:100F80001AC013968C911397811519F093818913C8
:100F900012C015968C911597811519F095818913BA
:100FA0000AC014969C91911521F081E024812913A7
:100FB00003C080E001C081E081700895809101014B
:100FC00008952FB7F8946091D6017091D701809160
:100FD000D8019091D9012FBF0895CF92DF92EF925F
:100FE000FF92CF93DF93D82FC92FC0908704D09062
:100FF0008804E0908904F0908A04E3DF6C197D098D
:101000008E099F09643F71408105910510F1D9DF78
:101010006B017C0182E390E0A0E0B0E0C09252025C
:10102000D0925302E0925402F092550280934E0205
:1010300090934F02A0935002B0935102D093850435
:10104000C0938604DF91CF91FF90EF90DF90CF9017
:10105000089584EF91E0A0E0B0E0E0CF0895FC01B6
:101060009B018091CC019091CD018617970740F0AC
:10107000672B29F48091E8008E778093E800C901FE
:1010800040E0009741F4411106C08091E80082FFE2
:101090002FC080E00895209184032115A9F1253007
:1010A000A9F12091E80023FD2DC02091E80022FD48
:1010B000ECCF2091E80020FFE4CF3091F3002091A5
:1010C000F200009719F02830310558F041E028303F
:1010D000310509F040E02091E8002E772093E800E8
:1010E000D0CF41914093F10001972F5F3F4FE9CF5F
:1010F00080918403811541F0853041F08091E800B2
:1011000083FFC3CF81E0089582E0089583E00895CE
:101110008091C60187FF13C08091E80082FF06C05E
:101120008091E8008B778093E80008958091840394
:101130008111F2CF0895809184038115D9F38091B4
:10114000E80080FFF8CF8091E8008E77ECCF209107
:10115000E4003091E50095E6A9012091EC00822F92
:10116000817020FF06C08091E80080FF06C080E00B
:1011700008952091E80022FD1AC080918403811512
:1011800089F0853089F08091EB0085FD0FC02091BA
:10119000E4003091E50042175307F9F29A95E1F621
:1011A00084E0089582E0089583E0089581E0089541
:1011B000E8EDF0E080818E7F80831092E200109253
:1011C000DA001092E100A0EEB0E08C9181608C9387
:1011D00080818F77808319BCA7EDB0E08C918E7FE2
:1011E0008C9380818F7E80831092C5010895E09159
:1011F0008B03F0918C03309739F00284F385E02D56
:10120000309711F060E209950895982F9093E900C6
:10121000891771F07091EC002091ED005091F00071
:1012200021FD09C09F5F973089F78093E9000895F9
:10123000762F242F50E03091EB003E7F3093EB006F
:101240003091ED003D7F3093ED003091EB00316047
:101250003093EB007093EC002093ED005093F0007E
:101260002091EE0027FDDECF0895A0E0B0E0EBE393
:10127000F9E00C94AC31C8EDD0E088818F7E888392
:10128000E7EDF0E080818160808384E082BF81E0CF
:101290008093C50188818E7F888302EE10E0F8017B
:1012A00010821092DA0081EEC82ED12CF601108245
:1012B00088818F77888388818068888388818F7D03
:1012C000888319BC109284031092C40110924B02BF
:1012D0001092C30190EEE92EF12CF70180818B7FF3
:1012E000808388818160888342E060E080E08DDFD8
:1012F000F60180818E7F8083F80180818160808308
:10130000808188608083F70180818E7F80838881DF
:1013100080618883CDB7DEB7E8E00C94C831E091F6
:1013200096039091950329E0E91302C080E00895A7
:10133000AE2FB0E02E9FF0011124E956FC4F318111
:10134000361306C03081381303C03581341304C00E
:10135000FD013196E770E8CF81E0089581E0809348
:10136000CF054091CF055091D0056091D105709186
:10137000D2058FE090E00E946D3240E050E0BA016B
:1013800083E190E00C946D3281E08093E00080E294
:101390008093D8001092C9008FE097E20197F1F78F
:1013A00000C0000087E090EBDC018093D5059093AE
:1013B000D605A093D705B093D80588E19CE00FB679
:1013C000F894A895809360000FBE90936000FFCFC3
:1013D0000F931F93CF93DF938B01EA0190918403C6
:1013E000943051F58093E9008FEF9091E80095FDDE
:1013F00006C09AE69A95F1F700C08A95B1F78091F8
:10140000E80085FF19C0A3DE811111C08091E800BA
:1014100085FD06C08091E8008E778093E800F3CFC9
:10142000F80181918F018093F100219779F78091E4
:10143000E8008E778093E800DF91CF911F910F91A4
:101440000895792F603229F440E250E0682F82E05D
:10145000BFCF0895CF93DF93D82FC92F48E050E036
:10146000682F792F81E0B4DF88E0ED2FFC2FAEEC00
:10147000B1E001900D928A95E1F7DF91CF91089547
:10148000BC0146E050E084E0A3CFBC0143E050E063
:1014900084E09ECF9091CE0592FB222720F9281759
:1014A00071F080FB92F99093CE056091CD0570911B
:1014B000CE0584E090E00E94753282E0C0C90895B4
:1014C0001F93CF93DF93962F122F632F8430B0F4A6
:1014D000911114C0453090F4C42FD0E0CC0FDD1F23
:1014E0009AE0899FC00DD11D1124CE0189960E94DA
:1014F0005B32612FCE018A960E945B32DF91CF91E1
:101500001F910895CF9363E472E084EF93E029DDA7
:10151000C82F811519F084EF93E09ADC9091F503C0
:1015200086E0E4EFF3E0DF01282F1D922A95E9F72A
:101530009093F503A3E4B2E001900D928A95E1F750
:1015400081E0911101C080E08C2BCF910895A4E23D
:10155000B0E0EDEAFAE00C94A6314091F40350912A
:10156000F5036091F6037091F7038091F803909171
:10157000F9039CD42093F4033093F5034093F603CE
:101580005093F7036093F8037093F90386E0E4EF58
:10159000F3E0DE01179601900D928A95E1F7109124
:1015A000F70311951A8786E0FE013796DE011D9636
:1015B00001900D928A95E1F726E0FE013D96CE015D
:1015C0000196DC0101900D922A95E1F726E0FC01DD
:1015D000A4EFB3E001900D922A95E1F726E0E4EF45
:1015E000F3E0DE01179601900D922A95E1F726E0CF
:1015F000FE013796DE01539601900D922A95E1F790
:1016000026E0FE017396DC0101900D922A95E1F728
:1016100026E0FC01A4EFB3E001900D922A95E1F7DA
:1016200026E0E4EFF3E0DE015F9601900D922A954B
:10163000E1F76091F6032091FA03D82EE92EF0909D
:10164000F8030091F903211509F46DC0062E000C72
:10165000770B880B990B0E94283320E030E040E0A4
:101660005EE30E94B43320913E0230913F024091EC
:101670004002509141020E9491323B014C01612F86
:10168000110F770B880B990B0E94283320E030E074
:1016900040E05EE30E94B43320913A0230913B0275
:1016A00040913C0250913D020E9491325B01C82E54
:1016B000192FB301C4010E94F532062FB5018C2DFC
:1016C000912F0E94F532F62E602F002E000C770B22
:1016D000880B990B0E9428339B01AC01B301C40114
:1016E0000E94903260933E0270933F0280934002CA
:1016F000909341026F2D0F2C000C770B880B990BE8
:101700000E9428339B01AC01B5018C2D912F0E94C2
:10171000903260933A0270933B0280933C02909324
:101720003D0210E060E069A31AA3FBA20CA386E0CF
:10173000FE017F96DE01179601900D928A95E1F7E2
:1017400086E0FE013796AD2DBE2D01900D928A9553
:10175000E1F786E0ED2DFE2DDE01599601900D9208
:101760008A95E1F786E0FE017996DE0117960190F1
:101770000D928A95E1F786E0FE013796A4EFB3E07B
:1017800001900D928A95E1F786E0EEEEF3E0DE013E
:10179000179601900D928A95E1F78091F50398854F
:1017A000892B8093F503AEDE811102C08091420245
:1017B00010924202A496EEE00C94C2310F931F9354
:1017C000CF93DF93843008F561111FC04530E8F4F2
:1017D000C42FD0E0CC0FDD1F2AE0829FC00DD11DA9
:1017E0001124CE0189960E943A32082F10E0102F62
:1017F0000027CE018A960E943A329801282BC9010F
:10180000DF91CF911F910F91089580E090E0F8CF84
:10181000462F2091870330918803232B89F4703F52
:1018200039F4603F69F480918503909186030895AF
:10183000711106C0653020F4843010F460E0BECF32
:1018400080E090E00895A0E0B0E0E9E2FCE00C94D4
:10185000AD317C010091CC058091CB05082BC3E014
:10186000D0E010E0C8010C2E02C0959587950A942F
:10187000E2F780FD09C02197A8F7D12C8D2DCDB7B7
:10188000DEB7E7E00C94C931DC2EB7018C2FC0DF46
:10189000F7D8019781F3F2CF0F931F93CF93FC01F9
:1018A00087819085009789F4858100811181811558
:1018B00081F0611571F0C801C6DFC82F682FC8011B
:1018C0000E94B003B8018C2FA3DFCF911F910F911D
:1018D0000895C8010E94D403C82FF4CFCF93DF939B
:1018E000D82FC92FB0DF6D2F7C2F92DFC9D8DF91A1
:1018F000CF910895FC0184818115A9F0878190859D
:10190000009799F0BDD8282F92959F709630B9F026
:1019100080F4925F9F70923030F4203FD1F058F401
:1019200081E0283E58F080E0089580819181D6DFE3
:10193000EACF9A5FEFCF81E0243FA9F7089591E0C5
:10194000813F09F090E081E0283E08F080E0892B9B
:10195000089581E00895382F292FCB01A32FB22FAE
:101960008F3A22E09207A105B10520F48F5A9E4FCD
:101970000C943A3280E0089585E290E00E943A3279
:101980008B3689F486E290E00E943A32833C59F427
:1019900087E290E00E943A3291E0813909F090E0CC
:1019A000892F8170089580E0FCCFAAE0B0E0EBEDD4
:1019B000FCE00C94AC31C0908203D090830381E0B2
:1019C00090E0909383038093820310E082E0E82EFE
:1019D00083E0F82E00E021E030E0111104C0F701AF
:1019E000859195919C01402F60E0812F69DD0F5F0B
:1019F00082E0E80EF11C053071F71F5F143031F7FB
:101A00001A8219821C821B821E821D8218861F82E6
:101A100088EC90E09A87898701E610E0FE01319614
:101A20007F014AE050E0B801C7010E947932065FA9
:101A30001F4F013B1105A9F78AE0F70111928A9522
:101A4000E9F74AE050E0B801C7010E947932065F29
:101A50001F4F01301007A9F789E0F70111928A950D
:101A6000E9F78FEF9FEF9E838D8387E08A874AE0B7
:101A700050E0B801C7010E947932065F1F4F01355F
:101A8000F1E01F07A1F7D0928303C09282032A9648
:101A9000E8E00C94C831AAE0B0E0E1E5FDE00C9488
:101AA000AC31E0EEF1E080E5DF011D928A95E9F7C7
:101AB000ECE1F5E088E3DF011D928A95E9F780EE1D
:101AC000C82E81E0D82E7F0101EB10E0F701D18212
:101AD000C0824AE050E0B801CE0101960E942A324D
:101AE00088E0FE013196D60101900D928A95E1F7CA
:101AF00089859A85D70113969C938E931297BAE0A5
:101B0000CB0ED11CE7E0EE0EF11C065F1F4F01303B
:101B10001007E1F62A96E8E00C94C831AAE0B0E09C
:101B2000E4E9FDE00C94AA310AE014E0EE24E39429
:101B3000FE2C97E0B92E2FEDC22E21E0D22EAA2442
:101B4000A3944AE050E0B701CE0101960E942A32E8
:101B5000F8013896DF018B2D1D928A95E9F789816E
:101B60009A81D80111969C938E938F8112968C93B3
:101B700012978D8113968C931397888514968C9366
:101B80001497898515968C9315978B819C81179650
:101B90009C938E9316978A8587FD04C01E96DC92CF
:101BA000CE921D9780FF02C0F801A08681FF07C07A
:101BB000D80118969C911897926018969C9382FF72
:101BC00004C0F80190859460908783FF07C0D80116
:101BD00018969C911897986018969C9384FF04C05F
:101BE000F80190859061908785FF07C0D80118960D
:101BF0008C911897806218968C93BAE0EB0EF11CCA
:101C0000015F1F4FE1E5EE16E1E0FE0609F099CF16
:101C10002A96EAE00C94C631282FCB01283070F4C4
:101C20004AE0249F90011124B9016F597F4F4AE087
:101C300050E00E942A3280E090E008958FEF9FEFFD
:101C40000895AAE0B0E0E7E2FEE00C94B2319C0116
:101C500097558115914068F4BE016F5F7F4F822FC9
:101C6000DBDF892B31F489859A852A96E2E00C9492
:101C7000CE3188EC90E0F9CFA0E1B0E0E2E4FEE004
:101C80000C94A431FE01319680E1DF011D928A950A
:101C9000E9F70BE210E091E5A92EBB24B3942FEAFB
:101CA000422E22E0522E612C712C4F0173016201F1
:101CB000B1E14B165104610471041CF080E1C82E9F
:101CC000D12CA601B501C4010E944C32AC0CBD1C44
:101CD0000D2C000CEE08FF084C185D086E087F08FC
:101CE0000150104019F76096E0E10C94C0316FEF9D
:101CF00085E290E00E945B326FEF86E290E00E9406
:101D00005B326FEF87E290E00E945B3260E088E236
:101D100090E00E945B3249DEAFDF6BE685E290E047
:101D20000E945B3263EC86E290E00E945B3261E9E4
:101D300087E290E00C945B32CF9324E030E043E004
:101D400060E080E30E94FB30C82F811105C00E9433
:101D500070318C2FCF91089582E08A95F1F700C001
:101D6000F8CFCF93C82FE8DF8115C9F08C2F0E94E0
:101D70000D318FE391E00197F1F700C000000E9460
:101D80002531C82F92E09A95F1F700C00E9470317A
:101D900082E38A95F1F700C08C2FCF910895C0E0BF
:101DA000FBCFA2E0B0E0E7EDFEE00C94AF31182FDE
:101DB000F62EC2DF082F811106C000E0802F229688
:101DC000E5E00C94CB31103511F010923802106818
:101DD0001983FA8262E070E0CE0101960E943D31E3
:101DE000892B59F78DE58A95F1F700000E94703133
:101DF00081E291E00197F1F700C00000DFCF60E0E1
:101E00008436910550F067E784342FE2920728F476
:101E100064E670E00E94D93161508FE0C2CF0E9429
:101E200066308ADF811509F440C02AE62A95F1F769
:101E300000C00E9470318AE68A95F1F700C06AE519
:101E40008AE3AFDF811589F19FE728E381E09150B4
:101E500020408040E1F700C0000082E082DF83E0A4
:101E600080DF84E07EDF85E07CDF86E07ADF0E9431
:101E700070318FE19EE40197F1F700C000006FE040
:101E80008FE08FDF8FEC97E00197F1F700C0000043
:101E900060E080E186DF64E181E183DF62E083E688
:101EA00080DF80E05EDF8FE35CCF0895A8E1B0E0E3
:101EB000ECE5FFE00C94B0314B8B5C8B6D8B7E8B33
:101EC0008F8B988FFE01379686E0DF011D928A95F1
:101ED000E9F7809138028F01811108C060E080E548
:101EE00060DF811539F181E08093380225DF8115AB
:101EF00009F180E50E940D31BDE5BA95F1F70000CA
:101F000066E070E0C8010E9456318F8187708111B0
:101F1000109238020E94703189859A859195819539
:101F200091099A8789878B859C85919581959109DF
:101F30009C878B8786E0FE013796DE011196019023
:101F40000D928A95E1F786E0FE013196DE011D963D
:101F500001900D928A95E1F78D8583FD05C08981F9
:101F600087FD17C01092390286E0FE017396DE01EC
:101F7000179601900D928A95E1F72F813885498552
:101F80005A856B857C8580E090E06896E4E00C944F
:101F9000CC314B815C812D813E8180913902811150
:101FA00003C081E080933902842F403851054CF002
:101FB0008FE78D8B822F2038310544F08FE78E8B91
:101FC000D3CF40385F4FACF780E8F3CF20383F4F96
:101FD000B4F780E8F4CF1F921FB61F9211248F939D
:101FE0009F93AF93BF9380914A02811113C0809158
:101FF000D6019091D701A091D801B091D901419615
:10200000A11DB11D8093D6019093D701A093D80153
:10201000B093D901BF91AF919F918F911F901FBE37
:102020001F9018952FB7F8948091D6019091D70101
:10203000A091D801B091D9012FBF0895CF93DF931C
:10204000C091140580911605C82B80911305811548
:10205000F1F0E8DF20911A0530911B05821B930BEC
:102060008838934110F00E944204D091130520E07B
:1020700088EB91E0FC013081019631112F5F31E056
:102080008E3B9307B9F721110E944204CD2B80911A
:10209000090480958C2390910804892B8093B601C4
:1020A00048E050E06DE873E086EB91E00E94163264
:1020B000892BB9F088E0E6EBF1E0ADE8B3E0019000
:1020C0000D928A95E1F7E0918B03F0918C033097A4
:1020D00041F00280F381E02D309719F086EB91E01A
:1020E0000995DF91CF910895811531F090911405F4
:1020F000892B80931405A2CF0895811519F00E94B1
:102100003A049CCF0895811531F090911605892BE2
:102110008093160593CF0895811539F0809590919D
:10212000160589238093160589CF0895CF93DF93F1
:10213000EC014A855B856E857F850E9414079B8133
:102140009095809116058923809316058C810E94B5
:102150003A0474DF86E0FE0111928A95E9F7DF9177
:10216000CF910895CF93DF93EC018D8181FD16C04F
:1021700082608D83809116059B81892B8093160543
:10218000809114059C81892B8093140557DF488525
:1021900059856E857F85CE010E94140710920E0529
:1021A00010920D058D8180FD02C0CE01BFDFDF9151
:1021B000CF910895962F2091CE0522FF0FC0682F52
:1021C000660F660F660F692B609317050E949803D0
:1021D00029DF909319058093180508950C949803AE
:1021E00090911305292F2823211559F080958923D3
:1021F00080931305811531F015DF80931A059093B4
:102200001B05089580E090E0F8CF0CDF2091F003EB
:102210003091F103232B211521F080937A039093C1
:102220007B032091F2033091F303232B211521F03E
:1022300080937803909379038EEE93E00C942807B3
:10224000611509F45DC0E3E3E80FE33150F4F0E019
:10225000E75EFB4C0C9400320E94CF068195809380
:10226000F103D3CF0E94CF06FACF0E94CF0681950B
:102270008093F003F6CF0E94CF06FACF0E94EF06BC
:102280008093F203EECF0E94EF068195F9CF0E9472
:10229000EF0681958093F303E4CF0E94EF06FACF17
:1022A000282F215D330BA90121E030E001C0220F6E
:1022B0004A95EAF79091EF03922B9093EF034091A8
:1022C000F503815D21E030E0F90102C0EE0FFF1F50
:1022D0008A95E2F7CF01611509F48CC0842B8093B5
:1022E000F50310C98091ED0381608093ED03B9CFB0
:1022F0008091ED038260F9CF8091ED038460F5CF8A
:102300009091F003482F50E08D3C59F42091F10357
:1023100027FF0DC01092F10391110BC01092EC0336
:1023200008C08E3CB1F42091F10312169CF3911574
:10233000B1F09091F2032091F303922B911102C01E
:102340001092EB03415D51094830510508F4B7CFB5
:1023500088CF8F3C39F497FFEACF1092F003909129
:10236000F103DACF803D19F41916BCF3E0CF2091C8
:10237000F203893D29F41216D4F61092F203D7CF56
:102380008A3D19F427FFD3CFF8CF2091F3038B3D7B
:1023900029F427FFCCCF1092F303C9CF8C3D19F459
:1023A0001216CCF3C4CF2FE2280F283080F4FA01A4
:1023B000E15DF10921E030E001C0220FEA95EAF782
:1023C00020953091EF0323232093EF03B0CF20918A
:1023D000ED032E7F8D3D59F02091ED032D7F8E3D35
:1023E00031F08F3D09F0A3CF2091ED032B7F209397
:1023F000ED039DCF8095842372CFCF93C82F811595
:10240000A9F08CEF8C0F813A98F4E8EBF1E08EEBB9
:1024100091E02191C21709F43DC08E179F07C9F7BB
:102420006C2F86EB91E00E948B0708DECF91089518
:1024300080E28C0F883068F4C77021E030E001C082
:10244000220FCA95EAF780911405822B8093140518
:10245000ECCF8BE58C0F833038F42C2F2452330BC8
:10246000C9010E943B07E2CFE8E5EC0FEB3150F4E5
:10247000F0E0EE0FFF1FED58FE4F808191810E942A
:102480006307D4CF83E38C0F833180F661E08C2F18
:10249000D7DECCCF8C2F0E94A507D0DDC1CFCF9344
:1024A000DF93EC01805E9109089720F063E870E10A
:1024B000209711F464E770E1CE010E9489038C2F0C
:1024C0009CDFDF91CF910895811559F19CEF980F12
:1024D000913A18F40E94A507B1CD90E2980F983078
:1024E00050F4877091E001C0990F8A95EAF7892F1F
:1024F0000E943A04F1CF9BE5980F933020F480E0DE
:1025000090E00C943B0798E5980F9B3120F480E015
:1025100090E00C94630793E3980F933110F460E01C
:102520008FCE08951F93CF93DF93182FEB0165DFB4
:10253000209731F4812FC8DFDF91CF911F9108954B
:102540008FEC97E00197F1F700C000002197F0CFE2
:1025500060E570E0893311F060E070E0E3CFA0E067
:10256000B0E0E5EBF2E10C94AB31EC018881811530
:10257000D9F0813009F03FC08981813021F48A810E
:102580002396E6DFF3CF823021F48A81239635DF6C
:10259000EDCF833021F48A81239696DFE7CF843014
:1025A00041F022968111E2CFCDB7DEB7E9E00C947D
:1025B000C7318A81239620E030E09AE0682F60538B
:1025C000770BAB016A30710560F02115310551F3CD
:1025D000EFECF7E03197F1F700C00000215031092E
:1025E000F4CF929FB001939F700D11249A01260F92
:1025F000371F8991E3CFE82FF0E0E354FE4FB4900A
:10260000282F26952695269530E0F901E355FE4FB3
:10261000E4908770F12C082E02C0F594E7940A9498
:10262000E2F7E0FAEE24FF24E0F8F901E356FE4F6A
:10263000C490D12C082E02C0D594C7940A94E2F716
:10264000C0FACC24DD24C0F8F901E357FE4F049111
:1026500010E002C0159507958A95E2F701701127E1
:10266000E114F10411F081EEC8DEC114D10411F0BF
:1026700086EEC3DE60E070E08B2D54DFC114D10420
:1026800011F086EE21DFE114F10411F081EE1CDF80
:102690000115110511F08CE25BDF219667CF1F93C6
:1026A000CF93DF93182FA0918304B09184041097E7
:1026B00009F449C01092860410928504109209040E
:1026C000109208041696CD91DC911797CE019A9539
:1026D00081159F4108F4D07ED1E0C11101C0D0E046
:1026E0001996ED91FC911A97309731F01B966D91E8
:1026F0007C9180E00995D823D11539F08CEF8C0FAF
:10270000813A28F58C2F0E94A5071115A9F0E091B8
:102710008304F0918404808584FD0EC0809182043E
:10272000811551F0808191819C01215031092F3315
:102730003E4710F40E94ED0781DC10928404109251
:10274000830410928204DF91CF911F91089576DC6B
:102750008C2FBADEDACFCF9310921405C6E0E8EBE7
:10276000F1E0DF018C2F1D928A95E9F780E090E07F
:102770000E943B0780E090E00E94630710921605DC
:102780005DDCEEEEF3E0DF011D92CA95E9F71092F1
:10279000EC031092EB031092ED0337DDCF91089517
:1027A000DADF2FE78AE196E0215080409040E1F7A0
:1027B00000C0000088E19CE00FB6F894A8958093D3
:1027C00060000FBE90936000FFCFAAE2B0E0EBEE96
:1027D000F3E10C94B13186EC91E0FC01019620917B
:1027E000F100208321E08E3C9207B9F78091C70168
:1027F000893009F459C0C8F4823009F4B6C0833076
:1028000009F485C0813089F18091E80083FFEAC036
:102810008091C6019091C7019A3008F0E3C0E92F7A
:10282000F0E0E45DFB4C0C9400328A3009F48CC07B
:102830008B3051F78091C601813231F78091CA0106
:102840009091CB01892B01F78091E800877F8093DD
:10285000E8000E94880881E09091C801911101C0B0
:1028600080E08093020177DFCFCF8091C601813A6B
:1028700059F68091E800877F8093E8008091CA0133
:102880009091CB01892B61F060E080E090E070E0F6
:102890000E942F088091E8008B778093E800B4CFE6
:1028A00068E08EEC91E0F3CF8091C601813209F0AF
:1028B000ABCF8091CA019091CB018D7F892B09F01C
:1028C000A3CF8091E800877F8093E8008091E800A3
:1028D00082FF18C09091F3008091F200029731F4CA
:1028E0008091F100813011F0863021F48091F10067
:1028F000809301018091E8008B778093E8000E942B
:10290000880882CF809184038111E0CF7DCF8091B0
:10291000C601813A09F078CF8091CA019091CB012C
:10292000892B09F071CF8091E800877F8093E800C0
:102930008091E80080FFFCCF809102018093F1003C
:102940008091E8008E77D9CF8091C601813209F05D
:102950005BCF8091E800877F8093E8000E94880821
:102960008091C901809300014FCF8091C601813AC7
:1029700009F04ACF8091E800877F8093E80080913A
:10298000E80080FFFCCF80910001D8CF803889F02B
:10299000823841F58091CA018F70873018F5809395
:1029A000E9008091EB0085FB882780F91092E9000F
:1029B00006C080914B02880F9091C301892B9091A2
:1029C000E800977F9093E8008093F1001092F10067
:1029D0008091E8008E7723C0811116C08091C801D4
:1029E000813011F18091E80083FF0AC08091E800F6
:1029F000877F8093E8008091EB0080628093EB00FA
:102A0000AA96E3E00C94CD31823061F78091C80141
:102A1000811589F01092E9008091E800877F80930A
:102A2000E8000E948808DECF81E0933009F080E062
:102A300080934B02EFCF8091CA018F702FEF280F48
:102A4000263080F68093E9002091EB0020FFE2CF52
:102A5000933031F48091EB0080628093EB00DACF09
:102A60009091EB0090619093EB0021E030E0A901A0
:102A700002C0440F551F8A95E2F74093EA00109276
:102A8000EA008091EB008860E8CF8111ABCF109114
:102A9000C8011F778091E3008078812B8093E30049
:102AA0008091E800877F8093E8000E9488088091E9
:102AB000E80080FFFCCF8091E30080688093E30012
:102AC00083E0111101C082E0809384038BCF805892
:102AD000823008F087CF8091C8019091C9018C3D68
:102AE00053E0950799F583E08A838AE289834FB79B
:102AF000F894DE01139620E03EE051E2E32FF0E08F
:102B000050935700849120FF03C082958F703F5FE0
:102B10008F708A30C8F0895C90E08D939D932F5F11
:102B2000243161F74FBF8091E800877F8093E800F0
:102B30006AE270E0CE0101960E942F088091E800C1
:102B40008B778093E8004ECF805DE6CF292F332727
:102B50002330310509F44EC078F52130310509F4F0
:102B600088C08BE590E0EDE3F2E02230310509F01A
:102B700039CF2091E800277F2093E8002091CC01F5
:102B80003091CD018217930708F49C0140E0211594
:102B9000310509F073C0411171C08091E80082FDD8
:102BA000CDCF80918403811549F2853039F280912F
:102BB000E80083FFF2CFC2CF8091CA019091CB0190
:102BC0002132310509F446C02232310509F00ACF1D
:102BD0008330910508F006CFFC01EE0FFF1FE45D86
:102BE000FE4F0190F081E02D875D9E4FDC018C91BE
:102BF00090E010C09C013327823021F12330310551
:102C000068F4232BB9F4EEEFF2E0E4918E2F90E01C
:102C1000EEEFF2E0009709F4E5CEABCF23303105BB
:102C200009F0E0CEEAEAF2E0E4918E2F90E0EAEAE1
:102C3000F2E0F0CFEEEEF2E0E4918E2F90E0EEEED7
:102C4000F2E0E8CFE8ECF2E0E4918E2F90E0E8ECDF
:102C5000F2E0E0CF8330910508F0C4CEFC01EE0F26
:102C6000FF1FEE5CFE4F0190F081E02D89E090E0C7
:102C700080CF82E190E0E8E9F2E07BCF80918403AD
:102C8000811509F45BCF853009F458CF8091E800B5
:102C900083FD54CF8091E80082FD7FCF8091E800D2
:102CA00080FF75CF9091F3008091F20021153105DE
:102CB00019F08830910550F041E0089709F040E0A4
:102CC0008091E8008E778093E80061CF4491409333
:102CD000F1003196215031090196E8CF803809F092
:102CE00081CE8091E800877F8093E8008091C401C5
:102CF0008093F1006DCE811175CE1091C801123014
:102D000008F070CE8091E800877F8093E8001093F0
:102D1000C4010E9488081115F9F084E080938403AF
:102D200042E061EC81E00E94050942E261EC84E04E
:102D30000E94050942E261EC82E00E94050942E23C
:102D400060EC83E00E94050980918403843051F493
:102D500082E08093030146CE8091E30087FDDDCFC2
:102D600081E0DCCF81E0F5CFA0E0B0E0EAEBF6E176
:102D70000C94AD31162FD72FC42FD22E811599F078
:102D8000409311054FD99093C2018093C101C77040
:102D900081E001C0880FCA95EAF7A6D9CDB7DEB7A2
:102DA000E7E00C94C93190911105491333C0E090CC
:102DB000C101F090C20136D99C012E193F09790159
:102DC000812F9D2F0E94210EE816F90618F5D0E2FA
:102DD000DD0DCD1591F0C77011E0812F01C0880F76
:102DE000CA95EAF78AD9D83040F48D2D877001C092
:102DF000110F8A95EAF7812F77D9802FA9DBD83078
:102E000068F62D2D277081E001C0880F2A95EAF71A
:102E100074D9C4CFC77081E001C0880FCA95EAF7A2
:102E2000F7CFACE0B0E0E7E1F7E10C94A3317C012F
:102E3000DC0114968C91811509F4E2C161E0C701AF
:102E40000E944C0C8C01F7018581811529F180913C
:102E50000D0590910E050097F9F008171907E1F09C
:102E6000FC01FF27887F9927892B09F0A7C0A4E0E0
:102E7000EE0FFF1FAA95E1F7E357FB4F85818460B2
:102E8000858311830083CF016DD91092160561E00F
:102E9000C7010E944C0C8C01D7018C91813069F4E0
:102EA00011968C91811109C0BDD89093FD03809338
:102EB000FC03F70185818093FB03D70115968C9164
:102EC0000115BEE71B0709F07CC0811509F180914F
:102ED000CF0590E0019665E070E00E94D9318093C3
:102EE000CF054091CF055091D0056091D1057091EB
:102EF000D2058FE090E00E946D32E091CF05F0E0C6
:102F0000EE0FFF1FE755FE4F808191810E94FF0E5B
:102F1000D70115968C91811163C06801A7E5DA1A73
:102F2000C114B1E0DB0668F56EEF73E08C2D0E94F2
:102F30000C0E892B31F5C60154E0880F991F5A9564
:102F4000E1F7FC01E357FB4F2281213009F02FC14B
:102F50002091FE033091FF03232B99F02091000470
:102F600030910104232B69F0209102043091030475
:102F70004091040450910504242B352B232B09F494
:102F800020C1F7013580311409F43EC10E35FCE74C
:102F90001F0709F421C10F352CE7120751F00D3539
:102FA0003CE7130709F030C180911001811509F445
:102FB00013C11092100180E072DB11C1E0E0F0E07B
:102FC0005DCF0130EEE71E0709F0A2CF811509F4AD
:102FD0009FCF8091FA0391E089278093FA0398CFDD
:102FE000C80197578038910560F6003108F0F7C0A6
:102FF0006EEA72E080E090E00E94AB0C8111EFC0BD
:10300000812C912C5401011146C004E09E012F5FD8
:103010003F4F6901D601E02F1D92EA95E9F724019F
:103020003501FFEF4F1A5F0A6F0A7F0AC501B4012D
:103030000E94AB0C8983811509F4D1C0813009F05D
:10304000B3C0A50194012E5F3F4F4F4F5F4F2D83BB
:103050003E834F835887C301B2010E94AB0C182FE7
:103060008A83811509F4BBC08FEF810F833078F517
:103070006D817E818F8198850E94AB0C8B83811539
:1030800011F0C6016CDA2401350133E0430E511C06
:10309000611C711C19C0BFEA8B16B2E09B06A1042B
:1030A000B10409F49CC0C501B4010E94AB0CEFEF60
:1030B0008E1A9E0AAE0ABE0A8111EDCF0150A3CF2F
:1030C0004D805E806F80788453014201A3CF8BEFE7
:1030D000810F8330A0F52401350143E0440E511CDB
:1030E000611C711C6D817E818F8198850E94AB0C63
:1030F0008B83811549F3C301B2010E94AB0C8C8311
:10310000811108C02401350154E0450E511C611C99
:10311000711CDACF8B819C818130AFEF9A0710F060
:10312000982F8827163029F0173031F00E94062595
:10313000E9CF0E94B324E6CF0E94D424E3CF143019
:1031400009F0BECF6D817E818F8198850E94AB0C86
:10315000182F24013501B4E04B0E511C611C711C69
:10316000C501B4016D5F7F4F8F4F9F4F0E94AB0C25
:103170001115A9F1811599F18150990B4FEF489FD5
:103180009001499F300D1124E12FE150FF0B2E0FCC
:103190003F1F2150310908F497CF8FEC97E001973A
:1031A000F1F700C00000F5CFC601D9D98DCF22308C
:1031B00009F0E7CE2091020430910304232B09F497
:1031C000E0CEFC01EE56FB4F20812E7F20838357FB
:1031D0009B4F0E94B210D5CE81E080931001809168
:1031E00017058770811561F0D70115968C918115AF
:1031F00039F08091CE0582FF03C082E00E941F0457
:103200002C96E1E10C94BF3180911001811168C0CE
:10321000C80197558115914008F0FDC05801F8EF9D
:10322000AF22BB24A114B104D1F6F801FF2734E08A
:10323000EE0FFF1F3A95E1F79F0123573B4F6901BE
:10324000D70115968C91EE56FB4F908180FB90F93B
:103250009083811509F4D8C10E9412109093100533
:1032600080930F05F60182818F5F8283809116051E
:1032700090911405892B8383809113058483468163
:10328000578166857785C6010E941407D601159679
:103290008C9181FF5801B0920E05A0920D05D701C7
:1032A00015968C91811509F4A7C510921105980106
:1032B00030572332310508F088C584E090E00E9441
:1032C00047329093CE058093CD05F801E150F04749
:1032D000E232F10508F0E0C1EA5CFB4C0C940032EC
:1032E000380150EE651A710850901505809114054B
:1032F000582A80911305582A88E06816710408F04E
:103300005EC098012770332781E090E001C0880FEC
:103310002A95EAF7311409F44FC0582AD7018D9144
:103320009C910E94D40321E030E0F90102C0EE0F2D
:10333000FF1F8A95E2F7FE83ED832091830430918D
:1033400084043A87298740918B0450918C045C87D0
:103350004B874AE0C42E44E0D42EA12CB12C51104E
:1033600005C0D60112968C9181111BC0F601838194
:1033700090E02D813E8182239323892B91F08085DB
:10338000982F9770911101C087E038E0631671049F
:1033900008F065C0311409F45EC086958170811112
:1033A00063C09FEFA91AB90AAFE0CA0ED11CB8E0FA
:1033B000AB16B104A1F61CC080955822AFCF3110D6
:1033C00037C080918B0490918C040817190781F401
:1033D00010928C0410928B0410928704109288042F
:1033E0001092890410928A04109286041092850427
:1033F0008091830490918404009709F409CFE8E058
:103400006E16710408F0EBC0652D0E94A0068111B4
:1034100002C081E044D9F7018581F801E851FC47F9
:10342000E730F10508F03BCFE85AFB4C0C94003232
:1034300010938C0400938B040E94E107609387042F
:10344000709388048093890490938A041092860470
:103450001092850463CF82FB882780F9A0CF3114B6
:1034600009F49FCF80FF9DCFD6018D909C900815C9
:10347000190519F4311409F494CFE985FA85EC158E
:10348000FD0509F48ECFD6011D96ED91FC91309784
:1034900021F08081811509F484CF652DC6010E9439
:1034A000A006811509F47DCF81E00815190509F002
:1034B00080E0482E43208114910441F0411006C061
:1034C000EB85FC858E169F0609F06BCF80E0E7D870
:1034D000D0928404C092830481E0809382048FE0C0
:1034E0008A9DF0018B9DF00D1124E65FFB4F8581D5
:1034F0008093090441100EC08114910459F0808119
:1035000091819C0124503109213A310508F049C0CC
:103510000E94A5078FE08A9DF0018B9DF00D11247C
:10352000E65FFB4FC680D780C6019A9581159F4103
:1035300010F420EED22299249394C60101978F3380
:103540009E4708F0912C8FE08A9DD0018B9DB00D95
:103550001124A65FBB4F1996ED91FC911A973097F5
:1035600031F01B966D917C9181E009959822911420
:10357000A9F08FE08A9DF0018B9DF00D1124E65F8C
:10358000FB4F868197810E945F0380930804C601E8
:1035900048E06416710440F40E94ED070E941E107A
:1035A0000CC00E946412B6CF0497813A910558F47A
:1035B0006C2D86EB91E00E948B07411409F428CE14
:1035C0000E941E100CCE0E941E108FE19EE40197F7
:1035D000F1F700C000008C2D0E94FD11EECFDC0140
:1035E0002D913C910217130739F4311008C0109245
:1035F000820480E054D80CCE311409F409CEFC01C9
:10360000808585FD05CEF5CFF90144855585668514
:103610007785C9010E941407D60115968C9181FF08
:103620003ECEC6010E94961080910D0590910E0528
:103630000817190709F033CE10920E0510920D05E8
:103640002ECE06E221EE41EE6AE17CE78DDBC7CDAE
:1036500007E225EE45EE6BE17CE7F8CF06E221EECE
:1036600040EE68E17CE7F2CF07E225EE44EE69E147
:103670007CE7ECCF06E221EE42EE6CE17CE7E6CFA0
:1036800007E225EE46EE6DE17CE7E0CF08E221E0BF
:1036900045EE6EE17CE7DACF8091CD0581608093C5
:1036A000CD056091CD057091CE0584E090E00E943B
:1036B000753251D894CD8091CE0588608093CE0527
:1036C000F0CF8091CD058260EACF8091CD058460F6
:1036D000E6CF8091CD058860E2CF8091CE058160F4
:1036E000EDCF8091CE058260E9CF8091CD058061DC
:1036F000D6CF8091CD058062D2CF8091CD058064F8
:10370000CECF29D88091CD058068C9CF8091CD05D5
:103710008C60C5CF8091CE058360D0CF8091CD05E0
:103720008E7FBDCF8091CE05877FC8CF8091CD059C
:103730008D7FB5CF8091CD058B7FB1CF8091CD05A9
:10374000877FADCF8091CE058E7FB8CF8091CE059B
:103750008D7FB4CF8091CD058F7EA1CF8091CD0597
:103760008F7D9DCF8091CD058F7B99CF0E94AB132C
:103770008091CD058F7793CF8091CD05837F8FCFBB
:103780008091CE058C7F9ACF8091CD05992782FFBD
:10379000939590FB82F990FB83F981CF8091CE05C0
:1037A000982F909590FB80F990FB81F987CF9091AD
:1037B000CD05892F8F7B96FF806471CF0E94AB135C
:1037C0009091CD05892F97FB87F9805868CF61E0EC
:1037D0008EE090E00E945B3264CF60E0F9CF909180
:1037E000CD05892F8F7E94FF806159CF9091CD05B3
:1037F000892F8E7F90FF816052CF9091CE05892FC7
:10380000877F93FF88605ACF89E201C30737BCE7FF
:103810001B07F9F00837ECE71E0751F19801205E0D
:1038200032452032310550F581113FC00F7181E0E2
:1038300090E09C0102C0220F331F0A95E2F7890134
:10384000622F83E090E00E945B32802F0E949203FF
:10385000C6CC811549F081E00E94980343E062E004
:1038600081E00E94F603BBCC81E00E94A203F6CF68
:10387000811511F082E0F0CF82E0F7CF8115A9F039
:103880000A353CE7130709F476C008F04EC0013052
:103890005CE7150709F46DC003308CE7180709F4DD
:1038A00062C001151C4709F451C0F701878190855A
:1038B000009709F464C00E9440058C01F701B580AF
:1038C000A680A2942FE0A22280911705877081150F
:1038D00001F1CB2CB114F1F0812F807F803461F0A5
:1038E00080E2800F8830A8F0812F807E803221F422
:1038F000023078F0A11469F08091CE0582FF09C0F2
:1039000082E00E941F04809117058770CC24C39425
:103910008111C12CE12FE295EF70103C08F0A5C099
:10392000F0E0E15AFB4C0C9400320B35ACE71A077F
:1039300021F18091CE05002482FF0394802D0C3567
:103940001C4709F0B2CF0E944A0AAFCF0E94AB13C6
:10395000EFE7FAE126E0E150F0402040E1F700C057
:1039600000000E94C4096FEF7FEF80E090E00E94AA
:1039700075320E94D01381E0E6CF80E0E4CF8581EC
:10398000C080D180811569F0C6010E94230C182FD8
:10399000682FC6010E94B003B601812F0E94080C57
:1039A0008ACFC6010E94D403182FF6CFF12FFF70E3
:1039B000DF2E103118F0D29490EFD922B114B9F063
:1039C000D11469F080E2800F883010F0011109C035
:1039D000809114058D29809314050E941E10802F5C
:1039E00042C0809116058D2980931605F6CF802F51
:1039F0000E946412D114C9F180E2800F883010F067
:103A0000011104C08D2D0E943A0406C0D09480910B
:103A100016058D21809316050E941E1026C0212FA9
:103A20002F70D22E107F103219F0D29480EFD8224E
:103A3000011549F0013009F484C0B11409F490C0B3
:103A4000A114B1F1CCCF8091CE0582FD2DC0B1146F
:103A500029F1D11439F0809114058D298093140532
:103A60000E941E1080E00E94FD11C11409F4D8C00C
:103A70008091170580FDD4C0D70115961C928695BC
:103A8000869586950E949803C701CBD9809117052A
:103A90008695869586950E94A203C2C080E00E940A
:103AA0006412D11411F3AECFB11469F1A11004C0A6
:103AB0008D2D0E947410D9CF31E0A31210C0109147
:103AC00013058D2D8123D81681F20E941210909338
:103AD0001B0580931A051D2910931305C6CF45E0D9
:103AE000A412C3CF8D2D0E9474108D2D0E94F01052
:103AF000809115059D2D9823D91609F4B6CF8D29EF
:103B000080931505B2CFA11012C08D2D0E947D109B
:103B10008D2D0E94F010809115059D2D98239115F3
:103B200009F4A3CFD094D822D09215059ECF51E0AE
:103B3000A5129BCF809114058D21811509F495CF95
:103B4000E4CFB11429F086E0A81608F08ECFB0CFEC
:103B500095E0A91608F089CF8D2D0E947D1085CFA4
:103B6000A114D1F3093349F4AFEFB3EFE1E0A15071
:103B7000B040E040E1F700C00000802F0E946412D6
:103B800074CF812F869586958370811561F0813081
:103B900009F06BCFC8019370B11002C080E090E0D3
:103BA0000E94630762CFC8019370B11002C080E029
:103BB00090E00E943B0759CF6B2D802F0E9420116F
:103BC00054CF812F8370811138C0B11027C0402F8E
:103BD000429546954770440F440F802F8F70042EF6
:103BE00001C0880F0A94EAF7202F207104FF07C054
:103BF0002FE030E001C0220F4A95EAF72095169594
:103C0000169513701230A1F0133081F03091CB056E
:103C1000113059F0822B83230E9492030E941907CE
:103C200060E0C7010E944C0CEBCA832B822BF4CFBF
:103C3000822B9091CB058927EFCFB11451F110FF62
:103C4000EDCF402F429546954770440F440F802F8B
:103C50008F70042E01C0880F0A94EAF7202F20717C
:103C600004FF07C02FE030E001C0220F4A95EAF7B9
:103C70002095169516951370123089F0133069F05F
:103C80003091CC05113041F0822B83230E949503A3
:103C9000C5CF823018F2D5CF832B822BF7CF822B62
:103CA0009091CC058927F2CF1F70B11439F0812F84
:103CB0000E949803802F0E947410B0CF802F0E9422
:103CC0007D10812F0E94A203A9CF023F71F170F4F1
:103CD000003FC9F0013F91F0B11409F465C0A1148F
:103CE00009F45FC0802F0E94FD1198CF033F21F19E
:103CF000043F91F78091CE0582FD2AC0812F8F71FC
:103D0000B11401F316C0B11469F0F5E0AF1608F074
:103D100085CF1F7181E090E0012E01C0880F0A94C9
:103D2000EAF7BECF26E0A216F2CF812F8F71B11035
:103D3000C9CF0E94980372CF80E0B11409F4A6CFD6
:103D40001F7181E0012E01C0880F0A94EAF79ECF0F
:103D5000B114C1F0809117058770843049F4109236
:103D600017051092190510921805812F8F71AACF8F
:103D700035E063E0A31608F051CF812F8F710E94C8
:103D8000DA104CCF45E0A41640F0109217051092BF
:103D900019051092180564E0F0CF81E00E941F041D
:103DA0003DCF812F8F71C5CFA114F9F2093349F4AA
:103DB0005FEF83EF91E0515080409040E1F700C009
:103DC0000000802F0E94641229CF0631BCE71B0738
:103DD00009F01CCD809114058A7A91E0811101C00F
:103DE00090E09093120565E3811101C069E286EBD2
:103DF00091E00E948B07E4CB0631ECE71E0709F047
:103E000005CD80911205811509F4FECC85E30E9451
:103E1000A507D6CBA0E0B0E0E0E1FFE10C94AD3126
:103E20008091E503803108F049C08091E403811559
:103E300009F444C0C091960389E0D82E809195037F
:103E40008C17E1F1EC2EF12CDC9EE0011124FE0137
:103E5000E956FC4F84818115B1F191818091E00395
:103E6000981331C090818091DF0398132CC0858115
:103E7000811129C0028113818091E1039091E203B5
:103E8000081B190B60E08FED93E00E944C0C0E9420
:103E9000210E08171907B8F48091E5038F7080612F
:103EA0008093E503C356DC4F88818F7080618883DF
:103EB0008FED93E00E9411170E941504CDB7DEB775
:103EC000E7E00C94C931E7012196C770B7CFAFE0A6
:103ED000B0E0EDE6FFE10C94A5318C0186E0F8013D
:103EE000DE011A9601900D928A95E1F7F801F580AE
:103EF000E4808FED882E83E0982E8091E30381117A
:103F000017C0E11491F0F11409F480C1C8010E94B6
:103F10007A0C811509F47AC189E0F801AFEDB3E0BC
:103F200001900D928A95E1F775DFFF24F3946AC042
:103F3000A280B380D090E4038091E1039091E203EA
:103F40003501681A790AD11409F411C1C080518071
:103F500060E08FED93E00E944C0C0E94210E6816E9
:103F6000790608F0B6C0E11401F38091E003F8018E
:103F70009181E090E503F0E1EF1608F064C098133A
:103F800020C09091DF03F801808198131AC020911E
:103F9000E6033091E703878190852817390789F474
:103FA000F1104BC08E2D8F7080618093E5038FEDF3
:103FB00093E00E9411178091E503F8018683F12CAC
:103FC00021C0F1103AC040E0652D8C2D0E948F0970
:103FD00040E0652D8C2D0E948F09F82E8111EFCFC6
:103FE0008A859B850E946E0C292F22952F70903414
:103FF00070F49F702230A0F09115B1F0F801968115
:10400000903190F48F2D2F96EFE00C94C1312A5F00
:104010002F70223068F0C8010E941117FD2CF2CFDA
:10402000911511F0811571F3805E883058F3F3CF4C
:10403000803F40F3815F8330F9CF8091E503816059
:104040008093E503BCCF98131EC09091DF03F80165
:104050008081981318C02091E6033091E70387818F
:1040600090852817390779F4F1100DC0E682C80150
:104070000E94111789E0F801AFEDB3E001900D92B5
:104080008A95E1F752CFC8010E947A0C811509F494
:10409000BDC0F11409F4BAC08091E503803208F480
:1040A0003BCF8091DF039091E0039A838983BC82A8
:1040B000AB828091E3038D831E82EF828091E603C1
:1040C0009091E70399878887CE0101960E94111786
:1040D00023CFD090E503F0E1DF1650F48FED93E0AD
:1040E0000E94111789E0F40111928A95E9F767CFD0
:1040F000E11409F41ACF9091E003F801818198133B
:104100001AC09091DF038081981315C02091E603B7
:104110003091E703878190852817390761F4F11002
:104120000AC0D682C8010E94111789E0F4011192D9
:104130008A95E9F7FACEC8010E947A0C811509F434
:1041400065C0F11409F462C08091E503803208F47F
:10415000E3CE8091DF039091E0039A838983BC8250
:10416000AB828091E3038D831E82DF82A7CF60E064
:104170008FED93E00E944C0C0E94210E6816790688
:1041800008F0B0CFE11409F4D0CEF11409F43EC028
:104190009091E003F801818198132EC09091DF0384
:1041A0008081981329C02091E6033091E70387812D
:1041B00090852817390701F58091E1039091E2037A
:1041C000A81AB90AF8ECAF16B10408F053CF8091E1
:1041D000E50380FD4FCF803108F44CCFF801868392
:1041E000982F907F903F09F442CF982F907F905F57
:1041F0008F70892B86833BCFC8010E947A0C811176
:104200008BCE8091E50381608093E503C8010E9415
:1042100011178BCEA2E1B0E0E0E1F1E20C94B031F5
:104220000A871B872C873D874E875F87688B798B32
:104230008A8BCE010A964BDE811128C0209195030E
:104240003091960389E0FE013A96DE0111960190C5
:104250000D928A95E1F78E858115C1F0822F90E04D
:1042600001968770992738171906D9F099E0929F1F
:10427000D0011124A956BC4FFE01319601900D9238
:104280009A95E1F7809395030E94150419E08091B7
:10429000960390919503891312C06296E4E00C9402
:1042A000CC310E94AB13109295031092960389E0D3
:1042B000EFEDF3E0DF011D928A95E9F7E7CF189F54
:1042C000C001112489569C4F02DE811531F3809183
:1042D000960390E001968770992780939603D7CF35
:1042E000EF92FF920F931F93CF93DF938091C805B6
:1042F000E091DE01CDE0811130C0CDB7DEB7E6E060
:104300000C94CA31D1E0DE0FD093DE01EE2EF12CF9
:10431000CE9FF0011124E05AFA4F84818115E1F01B
:1043200087819085892B21F481859285019651F4AE
:104330000081118122813381448155816681778199
:10434000808568DFCE9DF001CF9DF00D1124E05AED
:10435000FA4F148210921605ED2F8091C805E817C8
:1043600088F21092C8051092DE01C7CFA4E0B0E039
:10437000ECEBF1E20C94A33120915F05298397E0E7
:10438000992E01E010E02DE0322E34E0532E8824E7
:10439000839480915E059981891307C0A1DF0E94F3
:1043A00063062496E1E10C94BF319981892F90E056
:1043B0009C838B83FC01EE0FFF1FEC5AFA4F808128
:1043C0009181989ED001999EB00D1124FD01E45E6B
:1043D000FA4FFA83E983248121115BC06090C805FC
:1043E000E0E6F5E060E070E0712C661508F04FC083
:1043F000A384B484A981BA81CD90DC902FEF3FEFE4
:10440000412C442D50E07601E40CF11CE40CF11C2D
:10441000D701ED90FC90E114F10439F0AE14BF0423
:1044200009F0A90143949A01ECCF2F3F3207D1F153
:10443000D80102C0AA0FBB1F2A95E2F77A2A980179
:10444000042C02C0220F331F0A94E2F7A901415045
:1044500051097416150629F5369EF001379EF00DA8
:104460001124E05AFA4F989ED001999EB00D112464
:10447000A45EBA4F12962D913C91139730872783F3
:104480005482108211829287818715968C920E94A5
:1044900074068B819C8101969A83898383708983BA
:1044A00078CF14826F5F7F4F3D969FCF1092CA05E1
:1044B0001092C9051092110180915E0580935F05ED
:1044C0000E9463060DCFACE1B0E0E9E6F2E20C94A5
:1044D000A2314B8B5C8B6D8B7E8B8F8BB92E988F23
:1044E000A92E911110921605188A198A1A8A86E047
:1044F000FE017396DE011A9601900D928A95E1F7FE
:104500005F888091CE0582FF1FC00E94121020910B
:10451000180530911905821B930B8838934138F0A8
:104520008091170582FD03C082E00E941F040E9453
:10453000121020911A0530911B05821B930B8838AD
:10454000934110F00E9442045114D9F05E86BF8658
:1045500061E0CE010A960E944C0C61E0CE010A9601
:104560000E944C0C61E0CE010A960E944C0C4C015A
:1045700080356CE7960791F4A11419F181E08093DE
:1045800011015E86BF860A851B852C853D85452DDC
:104590005B2D688979898A893DDECDC081359C474C
:1045A00021F4A11471F082DFECCF82E588168CE74C
:1045B000980639F4A11429F0809111018111F3CFEB
:1045C000DDCF4CE1E42E45E0F42E412C612C712C22
:1045D000D7016D917C91CC24CA94DD24DA9480E0DB
:1045E000282F30E0FB01E80FF11DE80FF11D40819D
:1045F00051814115510539F08416950609F096014F
:104600008F5F6901EDCF10E0BFEFCB16DB0609F439
:104610004EC0F701448110911101411110E0D70102
:1046200015963C90159716969C911697A11409F42F
:1046300005C1111509F402C1311017C021E030E0A5
:104640000C2C01C0220F0A94EAF7922B16969C9329
:1046500020915C0530915D052233310530F422E371
:1046600030E030935D0520935C05E1E0F0E002C0AE
:10467000EE0FFF1F8A95E2F7CF010197D70116963B
:104680002C912817190699F4C090C905D090CA0535
:10469000C114D10409F453C00E9412108C199D0951
:1046A000C39708F44CC081E0F701848311E0412AEC
:1046B000BFEF6B1A7B0AE7E0EE0EF11CF8E06F1615
:1046C000710409F085CFA11409F417C1411409F44C
:1046D00014C10E9412109093CA058093C90580915D
:1046E000C805883040F591E0980F9093C80599E08F
:1046F000FE013A96DE01119601900D929A95E1F72E
:104700005D82BE822DE0829FC0011124805A9A4FA3
:1047100029E0FE013196DC0101900D922A95E1F726
:104720002FEF3FEFDC011A963C932E9319971C96BE
:104730009C928E921B976C96E2E10C94BE31209174
:104740005F0580915E05922FE0E0F0E001E0281720
:1047500009F448C0422F50E0FA01EE0FFF1FEC5A57
:10476000FA4F2080318037E0329DF001339DF00D0B
:104770001124E45EFA4F608171817C8F6B8FB0E011
:1047800030E0A0E0EB8DFC8DEA0FF11DEA0FF11D8A
:10479000C080D180C114D104E1F0F7010190F08113
:1047A000E02DFA8FE98F30E007C0E1E0C616D706AA
:1047B00009F0E0E0BE2B3F5FE98DFA8DE30FF11DBC
:1047C000E30FF11D608171816115710571F7AF5FB4
:1047D000D9CFB11581F13A17C8F4E1E0D7011496A9
:1047E000EC93F70190935F05EE15FF0509F45FCF99
:1047F00090E0FC01EE0FFF1FEC5AFA4F71826082CD
:1048000001968370992780935E0551CF37E0329DE2
:10481000F001339DF00D1124E45EFA4F0483EE1590
:10482000FF05F9F2291302C09F5F93709A012F5F71
:104830003F4F23708CCFE0E0F0E0F8CF292F30E03D
:10484000311024C061E070E002C0660F771F8A95C6
:10485000E2F7CB0101972817390791F010E0E1E06A
:10486000F0E002C0EE0FFF1FCA94E2F76F01C094A0
:10487000D70116968C9116978C2116968C9317CF8C
:10488000411569F3C3010E947406E8CFA9010C2CFD
:1048900002C0559547950A94E2F7C9010197822312
:1048A0009323892B39F540FF25C0D70112968D91AE
:1048B0009C91892BD1F087E0FE013196DF011D929A
:1048C0008A95E9F70E9412109C018B839C8384E0F7
:1048D0008D83F70192818381792F98878987098158
:1048E0001A8144E05E816F8195DCD70115961C9298
:1048F000132DB5CF142F1170B2CF90915F05809119
:104900005E05981731F032DDB1E04B1609F413CF94
:1049100038CEE6DC1092CA051092C9050E946306E3
:10492000F3CFA6E0B0E0E7E9F4E20C94B0310E94E6
:1049300012108C018091890390918A03801791074E
:1049400071F019821A820E941210BC0149815A81A9
:1049500080E090E0B8DD10938A03009389032696E7
:10496000E4E00C94CC31A6E0B0E0E9EBF4E20C9486
:10497000B2319093860380938503811520E29207DC
:1049800030F40E944F122696E2E00C94CE3180EF74
:1049900089838A830E9412108160BC0149815A81F7
:1049A00081E091E090DDEFCFA6E0B0E0EAEDF4E247
:1049B0000C94B0318C01909386038093850301158C
:1049C00080E21807B0F4802F0E946412C801805E54
:1049D0009109089728F06CE870E10115110511F4B0
:1049E0006DE770E1C8010E9489032696E4E00C940B
:1049F000CC3180EF89838A830E9412108160BC01D0
:104A000049815A8181E090E05EDDEFCFCF93DF9363
:104A1000D82FC92FA8DF8D2F9C2FC6DFDF91CF9114
:104A200008950F931F93CF93DF938C01862F6EEF22
:104A300073E00E940C0E892B91F4C091FE03D0917B
:104A4000FF03209761F0F8018281833039F4CE01B1
:104A5000DDDFCE01DBDFCE01D9DF01C0E0F7DF9182
:104A6000CF911F910F9108950F931F93CF93DF93D1
:104A70008C01EB016EEF73E08C2F0E940C0E892BE2
:104A800009F057C0FE01FF27D80112968C911297AA
:104A9000E05DFD4F8130A9F415968C9182FD4EC0EA
:104AA00080FF4CC082E080838091000490910104DB
:104AB0000097B9F48091FE039091FF030097C9F12C
:104AC00010C08230A1F515968C9182FD26C080FD24
:104AD0000AC083E0808380910204909103040097D0
:104AE000F1F041DF26C084E080838091040490913E
:104AF00005040097B1F78091FE039091FF030097A2
:104B000001F184DF8091000490910104009749F73E
:104B10008091FE039091FF03E4CF85E08083809134
:104B2000FE039091FF03009721F070DFF1CF86E044
:104B30008083DF91CF911F910F91089581E0808351
:104B4000B9CF8091000490910104B8CF0F931F93C7
:104B5000CF93DF938C01EB016EEF73E08C2F0E94FB
:104B60000C0E892B71F4DD27C05DDD4F8881F801C3
:104B7000128218828330E9F048F4813059F0823093
:104B800081F0DF91CF911F910F9108958430B1F0A2
:104B90008530B9F78091FE039091FF03009789F368
:104BA00006C08091000490910104009799F3FCDE07
:104BB000E8CF8091020490910304F7CF8091040420
:104BC00090910504009799F72091FE033091FF031F
:104BD000809100049091010421153105F9F20097AC
:104BE00031F7C901E4CFCF93DF93A8E3B1E06DE3E0
:104BF00071E041E030E02D912F3F79F0E22FE29516
:104C0000EF70E05EF0E0808190E02F7002C095953B
:104C100087952A95E2F780FF22C080E0382B440F69
:104C20006A177B0741F78091490283131AC080916C
:104C3000C001811509F1C091BE01D091BF010E9450
:104C400012108C1B9D0B0597B8F080914902909132
:104C500081038913809381031092C0010DC0842FBA
:104C6000DDCF3093490281E08093C0010E94121091
:104C70009093BF018093BE01DF91CF910895CDB78E
:104C8000DEB7E0970FB6F894DEBF0FBECDBF85B795
:104C9000806885BF85B7806885BF84B7877F84BFFC
:104CA0000FB6F894A89580916000886180936000A9
:104CB000109260000FBE80E890E00FB6F8948093E9
:104CC0006100909361000FBE81E0809303018CE34B
:104CD00096E09093B5018093B4010E944B060E9428
:104CE0004B0D0E948E0D8AE0E5E1F1E0DE011196A8
:104CF00001900D928A95E1F7FE0131969E01255FA4
:104D00003F4FEFA7F8AB41E050E08191A82FA2956B
:104D1000AF70B0E091966C9191978F708A0102C04C
:104D2000000F111F8A95E2F7C801962F982B9196D4
:104D30009C93919792969C919297809589239296B5
:104D40008C93E217F30709F70E94D8080E943509EF
:104D50008091E20084608093E200789480918403E3
:104D6000811599F08091E9001091EC008F701795F2
:104D700011271795182B1092E9008091E80083FD08
:104D80000E94E5131F701093E90082E084BD93E058
:104D900095BD9DE797BD80936E000E94BC0C81116C
:104DA00002C00E94770EEFE6F3E088E0DF011D927B
:104DB0008A95E9F78098889884988C981092640373
:104DC00010926203109263038FEF93E09093DB02E3
:104DD0008093DA021092D9021092D8021092D70270
:104DE0001092D60210925902109258021092570255
:104DF0001092560210926C0310926B039093610311
:104E00008093600310925F0310925E0310925D0323
:104E100010925C031092DF021092DE021092DD020B
:104E20001092DC0210926A031092690310926803D8
:104E3000109267031092660310926503A8E3B1E035
:104E40002DE331E041E050E08D918F3FA1F0E82F5C
:104E5000E295EF70F0E061A18F708A0102C0000F4F
:104E6000111F8A95E2F7C801902F9095962391A380
:104E700092A1892B82A32A173B0731F71092810355
:104E80001092490280E090E00E944732833E9E4F9C
:104E900021F40E94BC0C81111DC063EE7EEF80E006
:104EA00090E00E94753260E082E090E00E945B3208
:104EB00081E08093CB0561E083E090E00E945B326B
:104EC00060E074E184E090E00E9475320E94770E09
:104ED0000E94AE0982E090E00E943A3280934C0238
:104EE00084E090E00E9447329093CE058093CD05F8
:104EF0007ADE8FE59AEE0197F1F700C0000073DECD
:104F00008091810383FF08C06FEF7FEF80E090E026
:104F10000E9475320E94C40983E090E00E943A32F8
:104F20000E9492030E940F0F8FE090E00E94423295
:104F30006093CF057093D0058093D1059093D205EF
:104F4000663010F00E94AE09E091CF05F0E0EE0F60
:104F5000FF1FE755FE4F808191810E94FF0E84E084
:104F600091E090938C0380938B0382E0282E33246E
:104F7000339480918403853049F480918403853093
:104F800009F434C10E94AB130E9419072CDE8091F2
:104F90004D02E09081038E11C6C6C3DC00918504EA
:104FA000109186040115110591F1C0905202D09024
:104FB0005302E0905402F09055020E94E1076C19F0
:104FC0007D098E099F09C0904E02D0904F02E0905B
:104FD0005002F09051026C157D058E059F05B8F0CA
:104FE000C8010E944F1210928604109285041092FC
:104FF00052021092530210925402109255021092D3
:105000004E0210924F021092500210925102E09004
:105010000D05F0900E05E114F10441F100910F052A
:10502000109110050E9412109C01201B310B890168
:10503000C7010E94210E80179107C0F420910D0531
:1050400030910E05C9019927287F3327232B09F0BA
:1050500019C114E0880F991F1A95E1F783579B4FE8
:10506000DC0115962C9122FF0E94B2108091110153
:10507000811511F10091C9051091CA05011511059D
:10508000D9F00E941210801B910B20915C05309189
:105090005D052817390780F490915F0580915E05C2
:1050A000981709F4F2C062D910925D0510925C0560
:1050B0001092CA051092C90580917703811551F0AD
:1050C00010927703809171038093720380916F0334
:1050D0008093700380EFF8D72C0184EFF5D73C0163
:1050E00080916C03811521F080916B0381112BC09D
:1050F000EBE6F3E0FF93EF932CE633E03F932F933F
:10510000E6E58E2EE2E09E2EF8E5AF2EF2E0BF2E11
:10511000AAE5CA2EA2E0DA2EB8E9EB2EB2E0FB2E09
:1051200006ED12E027ED32E048ED52E06AED72E064
:10513000C2010E94570290936803809367030F9007
:105140000F900F900F9080916A03811521F080914C
:10515000690381112BC069E673E07F936F93AAE620
:10516000B3E0BF93AF934CED842E42E0942E5EEDFE
:10517000A52E52E0B52E60EEC62E62E0D62E7EE160
:10518000E72E73E0F72E0CE513E02DE533E04EE556
:1051900053E060E673E0C3010E94570290936603F8
:1051A000809365030F900F900F900F9040916703CD
:1051B0005091680380916503909166032091640388
:1051C000211178C04416550608F067C068167906A4
:1051D00008F480C083E080936403809163038115A9
:1051E00009F478C01092630311E075C080918403C4
:1051F000843031F10E94A70A10924A02A8E1B0E07F
:10520000E0E40FB6F894A895A09360000FBEE09379
:10521000600083B7817F846083BF83B7816083BF71
:105220007894889583B78E7F83BF0FB6F894A8953E
:1052300080916000886180936000109260000FBED2
:10524000D2DC80918103811509F497CE80914B02C5
:10525000811509F492CE19BCF2E0F9BD09B400FE43
:10526000FDCF8091D8008F7D8093D8008091E000A1
:1052700082608093E0008091E00081FDFCCF0E947D
:10528000AB137BCE80E090E0EBCE2AD81092CA051B
:105290001092C9050E9463060FCF68167906D0F4F4
:1052A00030926403809162038115A1F01092620331
:1052B0001FEF11C0213009F079C04416550608F4DB
:1052C0006EC06816790630F0109264032093630371
:1052D0001092620310E0E090FC03F090FD030E9446
:1052E00012108E199F0984369105B0F1E0906D037C
:1052F000F0906E030E9412108E199F09059760F1BD
:105300008091FB03811128C0111531F18091710347
:1053100090E09C012F5F3F4F237033274091720331
:105320004217130699F081599C4F41E0113009F062
:1053300040E0479544274795DC0114964C93209311
:10534000710380916F038F5F80936F030E9412102F
:1053500090936E0380936D0380E01AED20917203A9
:1053600090917103921709F458C030E0F901ED589B
:10537000FC4F808187FB882780F92F5F3F4F237088
:10538000332720937203909170039F5F9093700373
:10539000B12FB81B8B2F0E94A81281E0DFCF6816B7
:1053A000790608F097CF2092640390CF223001F560
:1053B0004416550670F06816790608F08BCF3092C7
:1053C000640380916203811509F484CF1092620313
:1053D0000BCF6816790608F47DCF83E080936403D1
:1053E00080916303811509F475CF1092630360CF38
:1053F0004416550658F06816790608F46BCF1092DB
:105400006403309262031092630364CF68167906D6
:1054100008F060CF20926403F4CF81110E94E1076D
:105420000E94A70A81110E94E10786E0EEEEF3E0F8
:10543000AFA5B8A901900D928A95E1F71092F003FB
:105440001092F1031092F2031092F3038B819C816E
:10545000892B811509F443C000917A0310917B03D5
:105460000E9412109C01201B310B9091EC039115AE
:1054700009F454C42531310590F19F3F19F09F5F25
:105480009093EC031B81111559F00E94CF0691E017
:1054900011160CF09FEF899F802D11248093F0034B
:1054A0001C81111559F00E94CF0691E011160CF0E5
:1054B0009FEF899F802D11248093F1038091F00349
:1054C000811569F01091F103111549F00E94C10690
:1054D0008093F003812F0E94C1068093F1038D8198
:1054E0009E81892B811509F443C0009178031091A6
:1054F00079030E9412109C01201B310B9091EB0349
:10550000911509F406C42135310590F19F3F19F03A
:105510009F5F9093EB031D81111559F00E94EF06D8
:1055200091E011160CF09FEF899F802D112480933C
:10553000F2031E81111559F00E94EF0691E0111639
:105540000CF09FEF899F802D11248093F3038091AD
:10555000F203811569F01091F303111549F00E94CF
:10556000C1068093F203812F0E94C1068093F3034A
:105570006FA578A98EEE93E00E94B10781110CC04F
:105580008091F0039091F103892B9091F203892B84
:105590009091F303892B81110E94051186E0EFA5FC
:1055A000F8A9AEEEB3E001900D928A95E1F70E9462
:1055B000190790917C03891721F080937C030E9446
:1055C000E10780918403843009F0D3CC83E0809399
:1055D000E9008091E80082FFCCCC8091E80090E067
:1055E00085FF05C00E94A708811519F191E08091FF
:1055F000E8008B778093E800911509F4BACC00910C
:10560000870310918803E9810115110571F1EE3FBF
:1056100009F04DC08A81833020F08550833008F036
:1056200046C0EA81EE3008F042C0F0E0E559FB4C9C
:10563000E7C600E210E0FE0131967F018091E800AC
:1056400085FD0AC08091E8008B778093E8000E9476
:10565000A708811599F3CACF8091F100D7018D93E6
:105660007D010150104051F7C1CFE43148F4E115FC
:1056700049F0E150E33130F4F0E0E758FB4CC0C6AC
:10568000EE3F79F28FEF898312C01A8289E08B8313
:105690000EC08A81823081F08330B1F0813091F781
:1056A0000E94E107B3D66B837C838D839E83CE01FA
:1056B00001960E94F7085DCC88E290E0DBD61B8261
:1056C0001C821D828E83F3CF80918203909183038D
:1056D000892B69F380918103DACF8A81823091F638
:1056E0006B817C818D819E8191D688E290E0E3D6AA
:1056F000DECF4C816B818A810E94DE0B982789273F
:1057000098279E838D83D3CF2D813E8132272327F7
:1057100032274C816B818A810E94600AC8CF0E9427
:10572000D50CC5CF80E18A83C2CF82E08A838FEA1D
:10573000AECF8C818D3108F0BACF8A809B809824BF
:1057400089249824A12CB12C8E010F5F1F4F780162
:10575000E80EF11C0E151F0509F4A9CF80E0BFEA81
:105760008B16B2E09B06A104B10420F4C4018F5A49
:105770009E4F80D6F80184830F5F1F4FFFEF8F1A73
:105780009F0AAF0ABF0AE6CF8091820390918303FC
:10579000892B09F48CCF8C818D3108F088CF882E2D
:1057A000912CA12CB12CCA80DB80DC24CD24DC24FC
:1057B000E12CF12C8E010F5F1F4F412C512C320137
:1057C000481459046A047B0408F071CF2FEAC2160A
:1057D00022E0D206E104F10438F4D80114966C9169
:1057E000C6018F5A9E4F67D6BFEF4B1A5B0A6B0AF2
:1057F0007B0AEFEFCE1ADE0AEE0AFE0A0F5F1F4F9A
:10580000DFCF0E943C0E53CF84E08DCF8C818D3151
:1058100008F04DCF882E912CA12CB12CCA80DB80B2
:10582000DC24CD24DC24E12CF12C412C512C320140
:105830008E010B5F1F4F481459046A047B0408F063
:1058400036CF80E0F8E2CF16D104E104F10418F479
:10585000C60189960FD6D8018D938D01BFEF4B1AE3
:105860005B0A6B0A7B0AEFEFCE1ADE0AEE0AFE0A2B
:10587000E2CF2C81622E712C2D3108F018CF8A8155
:105880009B819827892798274C01A12CB12C88321D
:10589000910508F00CCF422F50E060E070E04BA77C
:1058A0005CA76DA77EA748E250E060E070E0481971
:1058B00059096A097B09421751056105710508F408
:1058C000F6CE2091820330918303232B09F03EC052
:1058D0007C0159E2E50EF11C80FBCC24DD24C0F8EC
:1058E00080FF0BC08896C6D59D8189279827892778
:1058F00081159C4711F48FEF8D838BA59CA5ADA5D9
:10590000BEA5880D991DAA1DBB1D80FF17C0830170
:105910000150110935E0432E512C4C0E5D1E400EF6
:10592000511EC701860D971DA5D5D2019C918115E9
:105930009C4719F48FEFF20180833801FE01319604
:10594000EC0DFD1D2FEFC614D70438F08E010F5F4C
:105950001F4FC12CD12C760124C0948185818115E3
:105960009C4711F42483258312E0C10ED11C32968A
:10597000EACF28E282169104A104B10430F4D801E0
:1059800014966C91C401899696D5BFEFCB1ADB0AA9
:10599000EB0AFB0AEFEF8E1A9E0AAE0ABE0A0F5FF1
:1059A0001F4F2BA53CA54DA55EA5C216D306E40648
:1059B000F506F8F27CCE8091820390918303892BC7
:1059C00009F475CECE0101960E94F7083FEF40E73B
:1059D00052E0315040405040E1F700C000009ACA08
:1059E00088E0E0E2F1E0DE01919601900D928A9567
:1059F000E1F7FE0132968FE1DF011D928A95E9F70A
:105A000086E0898388E07F96DE01159601900D92ED
:105A10008A95E1F74CCE80E3898381E08A831B82FB
:105A20001C8245CE8B819C81092E000CAA0BBB0BDE
:105A300025E0880F991FAA1FBB1F2A95D1F7AC013B
:105A4000BD01405E5F4F6F4F7F4F481759076A0790
:105A50007B0708F42CCE8033E1E09E07A105B10559
:105A600008F025CE4133F1E05F076105710520F0B4
:105A700040E351E060E070E0481B590BBC01645FFB
:105A80007C4FCE010196C9D412CE4AE150E06FEFAF
:105A900070E0CE010796D7D48091820389830A8370
:105AA0001B8283E08C831D8285E00CCE81E090E038
:105AB000909388038093870382E390E09093800320
:105AC00080937F030E94121090937E0380937D0346
:105AD000EECD0115110571F1D0908103E0907D03A9
:105AE000F0907E030E9412108E199F098536910551
:105AF00040F1D5FE26C0D3FE24C00E941210909320
:105B00007E0380937D0380917F03909180030197B2
:105B10009093800380937F03892B61F41092880314
:105B20001092870381E090E0909383038093820337
:105B300000E010E08091820389830A8380917F03D3
:105B4000A6CD82E390E09093800380937F03F2CF11
:105B50001092830310928203AACD40E250E06FEFCF
:105B600070E0CE0101966FD4A2CDEB81E73008F052
:105B70009ECDF0E0E457FB4C43C4FE0134968DE12A
:105B8000DF011D928A95E9F788E089838A837FCDBA
:105B90008C819AE0F92E8E010F5D1F4FF8012F2D99
:105BA00011922A95E9F7B8010E940C0E8983F80139
:105BB000DE01129601900D92FA94E1F778CD1C81E6
:105BC0008AE0FE013596DE01919601900D928A954C
:105BD000E1F789A19AA10E943E069AA389A38BA10D
:105BE0009CA10E943E069CA38BA38DA19EA10E9416
:105BF0003E069EA38DA38FA198A50E943E0698A75E
:105C00008FA38FEF183060F43AE0139FB001112496
:105C10006F597F4F4AE050E0CE0181966AD480E010
:105C200089830E944B0643CD2C816AE0CE01819688
:105C3000DC01E62F1D92EA95E9F7283008F044C010
:105C4000629FB00111246F547F4F4AE050E002D4AC
:105C500080E089838AE0FE01B196DE011296D6CEFD
:105C60001C818AE0FE013596DE01919601900D922D
:105C70008A95E1F789A59AA50E943E069AA789A769
:105C80008FEF183060F4FAE01F9FB00111246F54B9
:105C90007F4F4AE050E0CE0181962BD480E089838B
:105CA0000E944B0D04CD2C816AE0CE018196DC016F
:105CB000E62F1D92EA95E9F7283030F4629FB00193
:105CC00011246F5F7E4FC1CF8FEFC3CF1C818AE05D
:105CD000FE013596DE01919601900D928A95E1F7CD
:105CE0008BA19CA10E943E069CA38BA38FEF183032
:105CF00060F4FAE01F9FB00111246F5F7E4F4AE00D
:105D000050E0CE018196F5D380E089830E948E0D0C
:105D1000CECC2B30310508F0FBCB2ACC2B30310513
:105D200008F0ADCBDCCBF82EFE2400E011E08F2D87
:105D300081238115A9F009831A820E9412109C8385
:105D40008B833D8291E08E2D8123811101C090E0F3
:105D50009E8349815A816B817C818D810E9463225F
:105D60000F5F110F053019F7E0924D020E94E10715
:105D700015C978941F921FB61F9211248F939F9379
:105D8000AF93BF938091D6019091D701A091D80194
:105D9000B091D9010196A11DB11D8093D6019093B8
:105DA000D701A093D801B093D901BF91AF919F9132
:105DB0008F911F901FBE1F9018951F920F920FB6C4
:105DC0000F9211242F933F934F935F936F937F9381
:105DD0008F939F93AF93BF93EF93FF938091E100D5
:105DE00082FF09C08091E20082FF05C08091E1003E
:105DF0008B7F8093E1008091DA0080FF23C0809147
:105E0000D80080FF1FC08091DA008E7F8093DA0077
:105E10008091D90019BC80FFA6C082E089BD09B479
:105E200000FEFDCF81E0809384038091C501811144
:105E300009C00E94D8080E9435098091E200846060
:105E40008093E2008091E10080FF1AC08091E2001F
:105E500080FF16C08091E2008E7F8093E2008091E7
:105E6000E20080618093E2008091D800806280939C
:105E7000D80019BC85E08093840383E080930301FC
:105E80008091E10084FF2EC08091E20084FF2AC04F
:105E900019BC82E089BD09B400FEFDCF8091D80015
:105EA0008F7D8093D8008091E1008F7E8093E10008
:105EB0008091E2008F7E8093E2008091E200816019
:105EC0008093E2008091C401811509F451C084E0FF
:105ED0008093840380918403843009F051C082E070
:105EE000809303018091E10083FF2CC08091E20048
:105EF00083FF28C08091E100877F8093E10082E0EA
:105F0000809384031092C4018091E1008E7F80937E
:105F1000E1008091E2008E7F8093E2008091E200B8
:105F200080618093E20042E060E080E00E94050929
:105F30008091F00088608093F00081E080930301FD
:105F400080930201FF91EF91BF91AF919F918F914B
:105F50007F916F915F914F913F912F910F900FBE65
:105F60000F901F901895109284031092C5016ACF6C
:105F70008091E30087FF02C083E0AACF81E0A8CF31
:105F800081E0AECF1F920F920FB60F921124EF92C5
:105F9000FF920F931F932F933F934F935F936F93B2
:105FA0007F938F939F93AF93BF93CF93EF93FF9381
:105FB00009EE10E0F8018081C091EC008F70C79568
:105FC000CC27C795C82B108280EFE82EF12CF70163
:105FD0008081877F808378940E94E513F801108286
:105FE000F701808188608083CF70F801C083FF91C2
:105FF000EF91CF91BF91AF919F918F917F916F91D1
:106000005F914F913F912F911F910F91FF90EF90D2
:106010000F900FBE0F901F901895803F09F188F4E4
:10602000843901F140F48533F9F08633F9F0843393
:1060300039F583E208958639D9F0873909F582E286
:106040000895853FB9F030F4813FB1F0843FC1F449
:1060500084E00895863F91F0873F91F487E00895AA
:1060600080E0089580E2089584E2089585E208952D
:1060700081E2089585E0089581E0089586E008951D
:106080008FE1089595E890937A00982F9072906828
:1060900090937B008F7190911201892B80937C00EB
:1060A00080917A00806480937A0080917A0086FDE6
:1060B000FCCF809178002091790090917A009F77B1
:1060C00090937A00922F0895A8DFDCCF289A219A26
:1060D000229A23982B9880E58CBD0895FC0180912D
:1060E00014018F3F09F085C080818F3F09F481C082
:1060F0001092D4058181811519F080E28093D40536
:1061000092818091D405923009F44FC0933009F404
:1061100050C08460913009F449C08381948121E0AA
:1061200030E02817390708F446C08091D4052032A2
:10613000310509F456C008F041C02830310509F492
:106140004BC02031310509F44AC02230310509F431
:106150003FC08CB59091D405892B8CBD8091D3051F
:10616000811519F08DB581608DBD208120931401BA
:10617000458140931301E22FE295EF70A1E2AE0F4B
:10618000B0E03C912F7081E090E001C0880F2A952B
:10619000EAF7232F282B2C93EE5DF0E0908141113C
:1061A00025C0892B808381E0089588608093D40581
:1061B000B4CF8C60FBCF220F331FB3CF2034310517
:1061C00099F083602038310521F68093D405C1CF42
:1061D00081E08093D305BDCF91E09093D30581609A
:1061E000F4CF91E09093D3058260EFCF809589231F
:1061F000D9CF80E00895A6E0B0E0E0E0F1E3B2C0DE
:1062000089836A834B833D832C8381E08E83CE0117
:10621000019664DF2696E2E0C1C0CF93DF938EBD86
:106220000E941210EC010DB407FE05C08EB590E07F
:10623000DF91CF9108950E9412108C1B9D0B843624
:10624000910588F38EEF9FEFF3CFCF93DF931EBCC2
:106250000E941210EC010DB407FE05C08EB590E04F
:10626000DF91CF9108950E9412108C1B9D0B8436F4
:10627000910588F38EEF9FEFF3CF0F931F93CF938A
:10628000DF93EC018C01060F171FC017D10739F4FB
:1062900080E090E0DF91CF911F910F910895899157
:1062A000BCDF97FFF2CF8EEF9FEFF4CF0F931F93DA
:1062B000CF93DF93EC018C01060F171FC017D10796
:1062C00039F480E090E0DF91CF911F910F91089514
:1062D000BCDF97FD02C08993F1CF8EEF9FEFF3CF24
:1062E000209114012F3F51F1E22FE295EF70A1E2CE
:1062F000AE0FB0E03C912F7081E090E001C0880FBC
:106300002A95EAF7232F282B2C93EE5DF0E02091BD
:1063100013019081211599F0892B80838FEF809351
:1063200014018DB58E7F8DBD9CB58091D40580956F
:1063300089238CBD1092D4051092D30508958095C1
:106340008923EBCF2F923F924F925F926F927F9271
:106350008F929F92AF92BF92CF92DF92EF92FF9275
:106360000F931F93CF93DF93CDB7DEB7CA1BDB0B21
:106370000FB6F894DEBF0FBECDBF09942A883988C6
:1063800048885F846E847D848C849B84AA84B984CD
:10639000C884DF80EE80FD800C811B81AA81B981D9
:1063A000CE0FD11D0FB6F894DEBF0FBECDBFED01ED
:1063B0000895AA1BBB1B51E107C0AA1FBB1FA6174C
:1063C000B70710F0A61BB70B881F991F5A95A9F79E
:1063D00080959095BC01CD01089597FB072E16F48A
:1063E000009406D077FD08D0E4DF07FC05D03EF42A
:1063F000909581959F4F0895709561957F4F089571
:10640000EE0FFF1F0590F491E02D09946927962760
:1064100069277827872778270895FB01DC0102C0C8
:1064200005900D9241505040D8F70895FB01DC01D2
:1064300004C08D910190801921F441505040C8F75B
:10644000881B990B0895DC0101C06D9341505040A9
:10645000E0F70895DC01CB01FC01F999FECF06C0FD
:10646000F2BDE1BDF89A319600B40D924150504012
:10647000B8F70895F999FECF92BD81BDF89A992792
:1064800080B50895A6E1B0E044E050E0E5CFA8E192
:10649000B0E042E050E0E0CFDC01A40FB51F415076
:1064A000504040F0CB01840F951F2E9105D04150F4
:1064B0005040D8F70895262FF999FECF92BD81BD9F
:1064C000F89A019700B4021639F01FBA20BD0FB632
:1064D000F894FA9AF99A0FBE08950396272FECDFE5
:1064E000EADF252FE9DF242FE7CF0196272FE4DF0E
:1064F000E2CFDC01CB0102C02D9105D041505040CC
:10650000D8F70895262FF999FECF1FBA92BD81BD05
:1065100020BD0FB6F894FA9AF99A0FBE0196089525
:106520005058BB27AA270ED0E5C0D6D030F0DBD01C
:1065300020F031F49F3F11F41EF4CBC00EF4E0952F
:10654000E7FBC1C0E92FE7D080F3BA1762077307F2
:106550008407950718F071F49EF5FFC00EF4E095DE
:106560000B2EBA2FA02D0B01B90190010C01CA010D
:10657000A0011124FF27591B99F0593F50F4503EB8
:1065800068F11A16F040A22F232F342F4427585FAA
:10659000F3CF469537952795A795F0405395C9F7C2
:1065A0007EF41F16BA0B620B730B840BBAF091507A
:1065B000A1F0FF0FBB1F661F771F881FC2F70EC019
:1065C000BA0F621F731F841F48F4879577956795EC
:1065D000B795F7959E3F08F0B3CF9395880F08F0D5
:1065E0009927EE0F97958795089504D06894B11177
:1065F000B5C0089598D088F09F5790F0B92F99278B
:10660000B751A0F0D1F0660F771F881F991F1AF0BD
:10661000BA95C9F712C0B13081F09FD0B1E00895AA
:106620009CC0672F782F8827B85F39F0B93FCCF32B
:10663000869577956795B395D9F73EF490958095B3
:10664000709561957F4F8F4F9F4F0895E89409C0D3
:1066500097FB3EF490958095709561957F4F8F4F95
:106660009F4F9923A9F0F92F96E9BB279395F695AB
:10667000879577956795B795F111F8CFFAF4BB0F29
:1066800011F460FF1BC06F5F7F4F8F4F9F4F16C08D
:10669000882311F096E911C0772321F09EE8872F17
:1066A000762F05C0662371F096E8862F70E060E0D3
:1066B0002AF09A95660F771F881FDAF7880F96954C
:1066C000879597F9089597F99F6780E870E060E0F3
:1066D00008959FEF80EC089500240A94161617067B
:1066E00018060906089500240A94121613061406C3
:1066F00005060895092E0394000C11F4882352F026
:10670000BB0F40F4BF2B11F460FF04C06F5F7F4FDD
:106710008F4F9F4F089557FD9058440F551F59F0C4
:106720005F3F71F04795880F97FB991F61F09F3F7E
:1067300079F087950895121613061406551FF2CFA7
:106740004695F1DF08C0161617061806991FF1CFF7
:1067500086957105610508940895E894BB2766271E
:106760007727CB0197F908950BD0C4CFB5DF28F078
:10677000BADF18F0952309F0A6CFABCF1124EECFE6
:10678000CADFA0F3959FD1F3950F50E0551F629F8C
:10679000F001729FBB27F00DB11D639FAA27F00D7A
:1067A000B11DAA1F649F6627B00DA11D661F829FA1
:1067B0002227B00DA11D621F739FB00DA11D621F86
:1067C000839FA00D611D221F749F3327A00D611DA3
:1067D000231F849F600D211D822F762F6A2F112485
:1067E0009F5750408AF0E1F088234AF0EE0FFF1FD8
:1067F000BB1F661F771F881F91505040A9F79E3F0F
:10680000510570F060CFAACF5F3FECF3983EDCF308
:10681000869577956795B795F795E7959F5FC1F74B
:10682000FE2B880F911D9695879597F90895F894FA
:10683000FFCF2C11321135113B1150115011501155
:10684000501150115011501150113E114311471168
:106850004D11721178117C11C614EC14F214EC1461
:10686000F21445156715F2146E167B168E1BF61B77
:10687000961B611B651B9A1B691B9E1BAA1B751B24
:10688000EF1B791BAE1B7D1BB21BD71B811BB61BDD
:10689000DE1B861BBC1BC41B6D1BA21B711BA61B16
:1068A0008A1BC01BCE1BE71BED1B5B1B921BFD1B3A
:1068B0002E1B341B211B281B3A1B401B461BD61CBE
:1068C000D61C0F1D0F1DC11DDC1D351D351DE11D05
:1068D000541E651E651EF02C0B2D122D572B572BA9
:1068E000452D562D692DA82DAD2D572B572B572BE8
:1068F000B52D452B492B6D2B792B842B8F2B422BC0
:10690000422B422B422BDB2C922B952B992BC42B09
:10691000012C042C062C392CBD2DC82DDF2D142E56
:06692000302E532E662EFE
:1069260000000100DE072A0A2E08400A450A210A4D
:1069360001014001FF919334379667F6F5F3F700AE
:10694600EE5B21B355DF2BA60044227B49012701CC
:10695600AC004F02680288029492C63697E200E9BC
:1069660000EA00B500B600B700CD008301CC008A6E
:106976000192019401210223022402250226022704
:10698600022A02B300B4006F0070009F01CB019F82
:1069960002A002E200E900EA00B500B600B700CDA9
:1069A600008301CC008A0192019401210223022472
:1069B600022502260227022A02B300B4006F0070E5
:1069C600009F01CB019F02A00258028403B004403D
:0469D600066009004E
:00000001FF
